:020000040000fa
:080000000002040000000000f2
:020000040000fa
:100400000f6121000e7f24000e0188000000000013
:100410000c00070040a92000010020001100070087
:10042000000020000000e000020032000000020096
:1004300000000000b66c0200000000000040da007e
:100440000000fe004440a900401b21000000e00025
:100450000300320000002000a00188004440a800f2
:100460000000060091018800800078000000eb0089
:1004700015003700e280400032a0b4009101ba00bc
:10048000e280400032a0b4009102ba00e280400055
:1004900032a0b4000002eb00472bde00f507b200eb
:1004a000602ce10004003a000059eb008301e900f0
:1004b000fdff3e00040037006128e100010032002a
:1004c0000082eb00040007001101ba000200e00006
:1004d000e8ff3a00000006003159ba008301e90044
:1004e0000c0032002159ba008301e90008003200f3
:1004f0000400e00003003a00e280400032a0b400b3
:10050000f5ff370011d9ba008301e900faff3a007c
:100510008100e800e180400032a0b4000000060045
:1005200000000000000000000000000000000000cb
:1005300000000000000000000040da000000fe00a3
:10054000839f68000100e00002003d006000100091
:10055000e08018000300e00002003d00600111008f
:10056000e0811900050007004f00e00002003b0099
:1005700060001000e0801800000006006022b80053
:10058000060220000000d0008180d2000482d20048
:100590008582d2000000a0000202520083825a002d
:1005a000030031000202420083824a000000a100e1
:1005b0000603e900f3ff3a0000000600889fbe0032
:1005c0008a9fbe008c9fbe0000017800c1d520002c
:1005d0001100e0000b003a0000d62000e06a88001d
:1005e000c06a8800016b8800d16a880021409000b1
:1005f0000004a000a0409800614090000004a0000a
:10060000e0409800e7004100c208de00c20cdd00b7
:10061000d46a80000de12000006121000d0550002a
:1006200022002000811f7800110009000205d80077
:1006300000067800cf007800c308dd00e4854000a4
:100640008001eb0006e12000c5d520000100370045
:1006500001027800244090000008a300020032004c
:100660000a003700110a78009400780021409000b9
:100670000008a300fbff320009014200828f5000f6
:1006800002003900840f51004600310094007800c8
:10069000848f5000eeff3e00868f5000020039002c
:1006a000858f5000eaff3900c06a8000800f520039
:1006b0004f003a00858f50004d003a008301e8005a
:1006c000e18f5100e2ff36008c8f540004003600a9
:1006d0008a8f5400020031000b04780012003700aa
:1006e000614ab8006151b900b0ff2f00010020003d
:1006f0000200500083805800800f5200818f5a0002
:100700000200350009047800070037000d8054000e
:100710003261210002004000110009000a80d80067
:100720000a80b90000047800080078006f00070014
:1007300080017800e10f40002d003200c06a800087
:1007400003087800c26a800064004100a240900063
:10075000808f5100020032000104a0000100370028
:100760000104a1002141980008804100640050006c
:1007700080097800c06a8800c2d52000020878008d
:10078000c16a8000214090000004a000a0409800b1
:10079000234090000004a100a041980002027800cc
:1007a000a7ff3700d26a8800828f50000900360008
:1007b0009200780060d52000a241900003487800a4
:1007c000a16a8800140978008040eb00d06a80009c
:1007d00021409800d06a8000000a780024409000f0
:1007e0000004a0002042980064004200010037008d
:1007f0000000eb004f06be004f05be004f04be00d8
:100800000000060064005000d06a8800a0409000fc
:100810000104a1002140980000000600889fbe004e
:100820008a9fbe0000057800e4015000130010000c
:10083000c285de00234090000008a30004003200bf
:10084000d36a8800234090000004a100a0419800d2
:100850000100780059ff0700000478000000e00064
:10086000170032008a0f50001500320060b8970060
:1008700008005000c284de00898f55000100360058
:10088000890578004259dd008a0078000800780068
:100890000f0007008a0f5400090031004248dd00b4
:1008a000000044008a0f5000050036000a00500086
:1008b00000004400a26a8000b36a80000288be0083
:1008c000080078004f05be004f04be00000006007f
:1008d0008001eb000200370061f079008301e8003d
:1008e000828f5100fcff3a0000000600889fbe0086
:1008f00080047800206b80000000e00003003a00d4
:10090000100007000000e0000a003500206b8000a6
:100910000900e00002003a000004780006003700f9
:100920000004780009004000060007000000e00015
:1009300001003d000084eb00080078004f04be0079
:1009400000000600800078000000e00004003a008b
:1009500000e12000206b88000101780006003700cc
:100960000081eb0000612100808f500002003e00fa
:10097000216b88000001eb000200780000000600f7
:020000040000fa
:020000040001f9
:0457f800fe4300006c
:020000040000fa
:020000040001f9
:0457fc007f3e0000ec
:020000040000fa
:100008009c0200009c020000e66f00000a700000dd
:100018002e7000009c0200009c0200009c02000060
:100028009c0200009c0200009c0200009c02000050
:100038009c0200009c0200009c0200009c02000040
:10004800225c00009c020000006f00009c0200007f
:100058009c0200009c0200009c0200009c02000020
:100068009c0200009c0200009c0200009c02000010
:10007800a66f00009c0200009c0200009c02000089
:100088009c0200009c0200009c020000a06e000080
:100098009c0200009c0200009c0200009c020000e0
:1000a8009c0200009c0200009c0200009c020000d0
:1000b8009c0200009c0200009c0200009c020000c0
:1000c8009c0200009c0200009c0200009c020000b0
:1000d8009c0200009c0200009c0200009c020000a0
:1000e8009c0200009c0200009c0200009c02000090
:1000f8009c0200009c0200009c0200009c02000080
:100108009c0200009c0200009c0200009c0200006f
:100118009c0200009c0200009c0200009c0200005f
:100128009c0200009c0200009c0200009c0200004f
:100138009c0200009c0200009c0200009c0200003f
:100148009c0200009c0200009c0200009c0200002f
:100158009c0200009c0200009c0200009c0200001f
:100168009c0200009c0200009c0200009c0200000f
:100178009c0200009c020000e24200009c02000079
:100188009c0200009c0200009c0200009c020000ef
:100198009c0200009c0200009c0200009c020000df
:1001a8009c0200009c0200009c0200009c020000cf
:1001b8009c0200009c0200009c0200009c020000bf
:1001c8009c0200009c0200009c0200009c020000af
:1001d8009c0200009c0200009c0200009c0200009f
:1001e8009c0200009c0200009c0200009c0200008f
:0801f8009c0200009c020000c3
:020000040000fa
:100208009c0200009c020000e66f00000a700000db
:100218002e7000009c0200009c0200009c0200005e
:100228009c0200009c0200009c0200009c0200004e
:100238009c0200009c0200009c0200009c0200003e
:10024800225c00009c020000006f00009c0200007d
:100258009c0200009c0200009c0200009c0200001e
:100268009c0200009c0200009c0200009c0200000e
:10027800a66f00009c0200009c0200009c02000087
:100288009c0200009c0200009c020000a06e00007e
:100298009c0200009c0200009c0200009c020000de
:1002a8009c0200009c0200009c0200009c020000ce
:1002b8009c0200009c0200009c0200009c020000be
:1002c8009c0200009c0200009c0200009c020000ae
:1002d8009c0200009c0200009c0200009c0200009e
:1002e8009c0200009c0200009c0200009c0200008e
:1002f8009c0200009c0200009c0200009c0200007e
:100308009c0200009c0200009c0200009c0200006d
:100318009c0200009c0200009c0200009c0200005d
:100328009c0200009c0200009c0200009c0200004d
:100338009c0200009c0200009c0200009c0200003d
:100348009c0200009c0200009c0200009c0200002d
:100358009c0200009c0200009c0200009c0200001d
:100368009c0200009c0200009c0200009c0200000d
:100378009c0200009c020000e24200009c02000077
:100388009c0200009c0200009c0200009c020000ed
:100398009c0200009c0200009c0200009c020000dd
:1003a8009c0200009c0200009c0200009c020000cd
:1003b8009c0200009c0200009c0200009c020000bd
:1003c8009c0200009c0200009c0200009c020000ad
:1003d8009c0200009c0200009c0200009c0200009d
:1003e8009c0200009c0200009c0200009c0200008d
:0803f8009c0200009c020000c1
:020000040000fa
:1028000054650000737400002043000061730000f1
:10281000653a0000200000000a0d0000002a0000b8
:102820002a2a000052650000736500007420000031
:102830005374000061740000657300002e2a0000cc
:102840002a2a00000a0d0000005500004152000035
:1028500054200000496e00006974000069610000a6
:102860006c6900007a650000642f00002e0a0000e9
:102870000d00000052650000736500007420000028
:10288000537400006174000065730000206f000045
:102890006e200000496e0000697400002e0a0000de
:1028a0000d000000476500006e65000072690000c1
:1028b00063200000646500006d6f0000206400006c
:1028c0006576000069630000652000006174000007
:1028d000746100006368000065640000202d000042
:1028e000207000006f6c00006c650000642c00001c
:1028f0002064000065760000696300006541000007
:102900006464000072650000737300003d00000005
:102910000d0a0000004300004d4400002063000049
:102920006f6d0000706c000065740000653a000077
:10293000200000005265000073650000742e000046
:102940000a0d0000005200006561000064200000d4
:10295000416400006472000065730000732e000083
:10296000204c00006f630000616c000020420000fa
:10297000445f000041440000445200003a2000003f
:10298000002e000020530000746f000072690000e8
:102990006e67000020610000646400007265000042
:1029a000737300002e0a00000d0000004c6f000041
:1029b000636100006c2000004e6100006d65000046
:1029c0002e0a00000d00000057720000697400001c
:1029d00065200000436c000061730000732e00004e
:1029e0000a0d0000005700007269000074650000c5
:1029f00020530000636100006e200000456e00005f
:102a0000616200006c6500002f44000069730000e3
:102a1000616200006c6500002e0a00000d000000dd
:102a20004f74000068650000722e00000a0d00005f
:102a3000005200006f6c0000652000004368000039
:102a4000616e0000676500002053000075630000a0
:102a50006365000073730000667500006c2e000053
:102a60000a0d0000005200006f6c0000652000009d
:102a700043680000616e00006765000020460000aa
:102a8000616900006c650000642e000020200000d9
:102a900045720000726f0000723a000020000000d2
:102aa000436f00006e6e00006563000074690000f3
:102ab0006f6e00002041000063630000657000003d
:102ac000746500006420000045760000656e00001b
:102ad000743a00002000000053750000636300009a
:102ae00065730000732e000020480000616e000036
:102af000646c0000652000003d20000000450000df
:102b0000727200006f7200003a200000004900005d
:102b10006e6300006f6d0000696e000067200000aa
:102b2000436f00006e6e0000656300007469000072
:102b30006f6e00003a200000526500006d6f0000cb
:102b4000746500005f420000645f000041640000a3
:102b500064720000203d000020000000436f000070
:102b60006d6d0000616e0000642000005374000071
:102b70006174000075730000204500007665000058
:102b80006e7400003a20000000500000656e0000e6
:102b9000646900006e6700002e00000045720000ae
:102ba000726f0000722000003078000030320000a8
:102bb0003a200000556e00006b6e00006f77000039
:102bc0006e200000436f00006e6e00006563000021
:102bd000746900006f6e000020490000442e000060
:102be00000450000727200006f7200002043000078
:102bf0006f640000653a0000004400006973000043
:102c0000636f00006e6e00006563000074200000ba
:102c100045760000656e0000743a00002000000058
:102c2000537500006363000065730000732e00009d
:102c300000450000727200006f7200002e0000005c
:102c400043490000443d000030780000303000006f
:102c5000303100002e200000004300006f640000af
:102c6000653d000030780000303200002e28000062
:102c7000436f00006e6e0000656300007469000021
:102c80006f6e00002052000065710000292e0000c8
:102c900000500000534d00003d300000783000002f
:102ca00030310000312e0000205300004349000065
:102cb000443d000000500000534d00003d30000036
:102cc0007830000030310000332e00002053000027
:102cd00043490000443d0000002100002121000084
:102ce00045720000726f0000723a00002050000030
:102cf000534d0000206e00006f7400002073000030
:102d000075700000706f0000727400006564000050
:102d10002e0a00000d000000436f000064650000f3
:102d20003d3000007830000034280000436f000080
:102d30006e660000696700002052000065710000a7
:102d4000292e00000a0d0000004800004944000040
:102d5000204300006f6e0000747200006f6c000072
:102d600020430000686100006e6e0000656c00008a
:102d70002e0a00000d000000484900004420000019
:102d8000446100007461000020430000686100009d
:102d90006e6e0000656c00002e0a00000d00000041
:102da0002121000021450000727200006f720000b6
:102db0003a200000556e00006b6e00006f77000037
:102dc0006e20000043680000616e00006e65000028
:102dd0006c200000494400002e0a00000d00000095
:102de000436f0000646500003d3000007830000053
:102df00035280000436f00006e6600006967000020
:102e00002052000065730000702900002e0a0000a7
:102e10000d00000044690000736300006f6e000045
:102e20006e65000063740000207200006571000090
:102e300075650000737400003a0000002044000033
:102e400041540000412e00000a0d00000020000047
:102e500043540000524c00002e0a00000d000000f8
:102e600044690000736300006f6e00006e6500002f
:102e7000637400002052000065730000706f000052
:102e80006e730000653a0000005700007269000090
:102e900074650000204300006c6100007373000043
:102ea00020450000727200006f7200003a2000009e
:102eb000002000002d200000414300004c200000b5
:102ec000636100006e6e00006f74000020620000fd
:102ed00065200000777200006974000074650000ce
:102ee0006e2000002a2a00002a2a00002a2a000058
:102ef0002a2a00002a2a00002a2a00002a2a000082
:102f00002a2a00002a2a00002a2a00002a2a000071
:102f10002a000000446500006d6f0000537400003b
:102f200061740000653a0000004800006369000019
:102f30005374000061740000653a000000650000f1
:102f40006e64000020640000656200007567000088
:102f50000a0d000000450000727200006f72000050
:102f60003a200000436100006e6e00006f740000a4
:102f700020660000696e000064200000636f00009e
:102f80007272000065630000742000007479000014
:102f9000706500002e0a00000d000000494e000080
:102fa000495400000a0d0000004800004349000099
:102fb0005f4300004d4400005f5200004553000095
:102fc000455400003a20000000480000434900003a
:102fd0005f4300004d4400005f5200004541000087
:102fe000445f0000424400005f4100004444000090
:102ff000523a00002000000048430000495f0000f2
:10300000434d0000445f00004c4f0000434100006e
:103010004c5f00004e4100004d4500003a2000008a
:1030200000480000434900005f4300004d44000099
:103030005f4300004c410000535300005f44000018
:103040004556000049430000453a000020000000ba
:1030500048430000495f0000434d0000445f00000a
:1030600053430000414e00005f4500004e41000008
:10307000424c0000453a0000200000004843000098
:10308000495f0000434d0000445f000041430000e1
:1030900043450000505400005f4900004e430000cb
:1030a0004f4d0000494e0000472e00002052000006
:1030b0004f4c00004520000043480000414e0000f6
:1030c00047450000205200004551000055450000d2
:1030d00053540000454400003a200000004800001e
:1030e000434900005f4300004d4400005f5300006f
:1030f000434100004e5f000044490000534100007e
:10310000424c0000453a00002000000053430000fc
:103110004944000020430000545200004c200000ad
:103120003d200000004c00003243000041500000f0
:103130005f4300004f4e00004e4500004354000026
:103140005f5200004553000050310000313a00004a
:10315000200000004c32000043410000505f00009e
:10316000434f00004e460000494700005f520000f8
:1031700045510000313100003a200000004c0000b1
:1031800032430000415000005f4300004f4e0000fa
:1031900046490000475f00005245000053500000c0
:1031a000313100003a200000005300004349000084
:1031b000442000004441000054410000203d000034
:1031c000200000004c32000043410000505f00002e
:1031d000434f00004e4e000045430000545f000086
:1031e0005245000053500000313300003a200000e7
:1031f000004c000032430000415000005f430000db
:103200004f4e000046490000475f00005245000055
:1032100051310000333a00002000000050530000fc
:10322000335f0000425400005f530000455400002b
:103230005f46000045410000545500005245000023
:103240005f4900004e490000543a00002000000091
:103250004c32000043410000505f00004449000030
:10326000534300004f4e00004e4500004354000001
:103270005f44000041540000415f000052450000df
:10328000535000003a200000004c00003243000080
:10329000415000005f44000049530000434f0000cc
:1032a0004e4e000045430000545f000043540000b0
:1032b000524c00005f52000045530000503a00009d
:1032c000200000004c32000043410000505f00002d
:1032d00044490000534300004f4e00004e4500009b
:1032e000435400005f44000041540000413a000094
:1032f0002000000048430000495f000044490000ee
:10330000534300004f4e00004e4500004354000060
:103310003a200000005500006e6b00006e6f000048
:10332000776e000020440000656d00006f200000f3
:103330005374000061740000652e00000a0d000047
:10334000005000006169000072200000436f00001f
:103350006e740000726f00006c6c000065720000fb
:103360002077000069740000682000006c61000094
:1033700073740000204200006c750000657400004a
:103380006f6f000074680000206400006f6e000022
:10339000676c0000652e00002e2e00000a0d000054
:1033a000004400006f6e0000652e00000a0d000052
:1033b000004400006576000069630000652000009d
:1033c000577200006974000065200000457200001b
:1033d000726f000072200000210d00000a00000042
:1033e000526500006164000020420000616300003b
:1033f0006b20000041440000445200002e0a0000ef
:103400000d000000496e0000697400006961000051
:103410006c6900007a650000204300006f6e0000b8
:10342000747200006f6c00006c650000722e00006a
:103430000a0d0000002000002d200000446500005f
:10344000766900006365000020520000656100009d
:103450006420000045720000726f000072200000be
:10346000210d00000a000000476500006e650000a5
:103470007269000063200000646500006d6f000049
:10348000206400006576000069630000652000008c
:1034900061740000746100006368000065640000ee
:1034a000202d000020650000766500006e7400008d
:1034b0002c20000064650000766900006365000050
:1034c000416400006472000065730000733d0000f9
:1034d00000470000656e000065720000696300002f
:1034e00020640000656d00006f200000646500002e
:1034f00076690000636500002064000065740000c8
:103500006163000068650000642000002d20000059
:1035100065760000656e0000740d00000a00000072
:103520000d0a00002a2a00002a2a00002a20000092
:10353000555300004220000045720000726f0000e9
:10354000722000002d2000006875000062730000ea
:103550002061000072650000206e00006f740000a2
:103560002073000075700000706f0000727400001e
:1035700065640000202a00002a2a00002a2a000090
:103580000d0a0000000d00000a2a00002a2a00008f
:103590002a2a000020550000534200002045000068
:1035a000727200006f720000202d00002064000085
:1035b0006576000069630000652000006973000003
:1035c000206e00006f740000207300007570000012
:1035d000706f00007274000065640000202a000013
:1035e0002a2a00002a2a00000d0a0000000d00000f
:1035f0000a2a00002a2a00002a2a0000205500007a
:103600005342000020450000727200006f720000fb
:10361000202d000020630000616e00006e6f00002e
:1036200074200000656e0000756d0000657200007a
:103630006174000065200000646500007669000088
:1036400063650000202a00002a2a00002a2a0000c0
:103650000d0a0000000d00000a2a00002a2a0000be
:103660002a2a000020550000534200002045000097
:10367000727200006f720000202d000020630000b5
:103680006c690000656e0000742000006472000028
:103690006976000065720000206900006e69000014
:1036a00074690000616c0000697a000061740000b8
:1036b000696f00006e20000065720000726f0000ec
:1036c000722000002a2a00002a2a00002a0d000089
:1036d0000a0000000d0a00002a2a00002a2a000021
:1036e0002a200000555300004220000045720000cf
:1036f000726f0000722000002d2000006f75000026
:10370000742000006f660000206800006561000002
:10371000702000006d6500006d6f00007279000080
:10372000202a00002a2a00002a2a00000d0a000090
:10373000000d00000a2a00002a2a00002a2a0000a0
:103740002055000053420000204500007272000026
:103750006f720000202d0000207500006e730000c5
:103760007065000063690000666900006564000020
:10377000202a00002a2a00002a2a00000d0a000040
:10378000000d00000a0d00000a53000065720000e1
:10379000766f0000536800006f6300006b2000002c
:1037a00046690000726d00007761000072650000dc
:1037b000205200006576000020000000322e00003c
:1037c000320000003a200000436f0000756c0000da
:1037d000642000006e6f000074200000696e00001d
:1037e00069740000696100006c6900007a6500007e
:1037f0002073000079730000746500006d2e0000d6
:1038000020200000486100006c740000696e000018
:10381000672e00000d0a00000d0a0000000d0000d8
:103820000a0d00000a2a00002a2a00002a2a0000a5
:103830002053000065720000766f0000536800009e
:103840006f6300006b20000046690000726d00008d
:10385000776100007265000020520000657600006c
:1038600020000000202a00002a2a00002a2a000046
:103870000d0a00000d0a000000200000436f000048
:10388000756c0000642000006e6f00007420000062
:10389000696e000069740000696100006c690000d5
:1038a0007a65000020550000534200002e200000e1
:1038b00020480000616c0000746900006e67000021
:1038c0002e0d00000a0d00000a00000043690000f0
:1038d00072630000756900007420000054650000e8
:1038e00073740000204d00006f640000652e00001e
:1038f0000a0d0000004400006566000061750000cc
:103900006c740000732000004c6f000061640000c4
:10391000656400002e0a00000d000000454500000f
:10392000505200004f4d0000205700007269000007
:103930007465000020450000727200006f72000084
:103940002e200000000a00000d45000072610000fa
:10395000736900006e67000020700000616700005e
:10396000652e00000a0d000000460000697200008c
:103970006d7700006172000065200000436f000059
:10398000646500003a200000000a00000d4c0000b1
:103990006f610000646900006e6700002053000042
:1039a000617600006564000020530000657400002b
:1039b000746900006e670000732e0000200a00008a
:1039c0000d000000496400006c65000020540000f8
:1039d000696d0000656f0000757400002e0a00001c
:1039e0000d0000005752000049540000455f0000e0
:1039f0005354000041540000453a000020000000ec
:103a000053740000616300006b4500007272000097
:103a10006f720000004d000061740000682000001b
:103a200045720000726f00007200000096010000f5
:103a3000a0010000aa010000b4010000be010000c6
:103a4000c8010000d2010000dc010000e601000016
:103a50007e080000940100009e010000a801000003
:103a6000b2010000bc010000c6010000d00100004e
:103a7000da010000e401000080080000900100006d
:103a80009a010000a4010000ae010000b80100008e
:103a9000c2010000cc010000d6010000e0010000de
:103aa000820800004c6f000061640000696e000035
:103ab000672000006465000066610000756c00000e
:103ac000742000007365000074740000696e0000cb
:103ad00067730000206600006f7200002000000085
:103ae0004c6f000061640000696e000067200000f8
:103af000616c00006c2000006465000066610000dd
:103b0000756c000074200000736500007474000080
:103b1000696e0000677300002e2e00002e0000006a
:103b2000446f00006e6500000a0d000000200000d8
:103b300045450000505200004f4d00002077000026
:103b40006f72000064730000207500007365000050
:103b5000642e00000a0d0000004c00006f610000a0
:103b6000646900006e670000207300006176000049
:103b70006564000020730000657400007469000033
:103b80006e670000732e00002e2e00000053000010
:103b900061760000696e0000672000005365000038
:103ba00074740000696e0000677300002e2e000020
:103bb0002e000000446f00006e6500002e0a000019
:103bc0000d000000456e0000746500007269000081
:103bd0006e670000204300006f6e00006669000001
:103be000672000004d6f0000646500003a0a000085
:103bf0000d0000004578000069740000696e000047
:103c000067200000436f00006e66000069670000d7
:103c1000204d00006f640000652e00000a0d0000ba
:103c2000005300005049000020420000757300005e
:103c3000204d00006f64000065200000300a000085
:103c40000d000000535000004920000042750000a4
:103c5000732000004d6f00006465000020310000fb
:103c60000a0d0000005300005049000020420000ef
:103c700075730000204d00006f6400006520000097
:103c8000320a00000d0000005350000049200000df
:103c900042750000732000004d6f00006465000055
:103ca000203300000a0d00000045000052520000c1
:103cb0004f520000205300005049000020420000f5
:103cc00055530000204d00004f440000450a0000fd
:103cd0000d000000496400006c65000020610000d8
:103ce000757400006f2d00006f66000066200000f4
:103cf0007365000074200000746f00002031000024
:103d0000302000006d6900006e2e00000a0d0000da
:103d100000490000646c000065200000617500002f
:103d2000746f00002d6f00006666000020640000c4
:103d300069730000616200006c650000642e000081
:103d40000a0d0000005400006f670000676c00005f
:103d500065640000206f000075740000707500003d
:103d60007473000020720000657300006574000029
:103d7000206f00006e200000646900007363000083
:103d80006f6e00006e650000637400002e0a000074
:103d90000d000000546f0000676700006c650000b4
:103da000642000006f7500007470000075740000de
:103db00073200000707200006573000065720000df
:103dc00076650000642000006f6e00002064000033
:103dd00069730000636f00006e6e00006563000091
:103de000742e00000a0d00000054000072690000eb
:103df0006d2000003d200000000a00000d000000c2
:103e0000505700004d200000467200006571000010
:103e1000756500006e630000792000003d20000001
:103e2000002000006b4800007a2e00000a0d000000
:103e30000053000065720000766f00002f4d0000f7
:103e40006f7400006f720000204600006f72000067
:103e500077610000726400002e0a00000d0000006f
:103e600053650000727600006f2f00004d6f000058
:103e7000746f00007220000052650000766500003b
:103e800072730000652e00000a0d00000041000062
:103e9000627300006f6c0000757400006520000004
:103ea000696e000070750000742000006d6f0000e6
:103eb000646500002e0a00000d000000526500003d
:103ec0006c610000746900007665000020690000e4
:103ed0006e70000075740000206d00006f640000bb
:103ee000652e00000a0d00000053000065720000fe
:103ef000766f000020530000696700006e610000cb
:103f00006c20000050650000726900006f640000c2
:103f1000203d000020000000206d0000732e0000f6
:103f20000a0d00000054000072690000676700007d
:103f300065720000204c0000696e00006b200000dc
:103f40004f6e00002e0a00000d00000054720000a9
:103f50006967000067650000722000004c6900007e
:103f60006e6b0000204f0000666600002e0a000005
:103f70000d0000004c650000667400002053000036
:103f800074690000636b0000204400006966000053
:103f900066650000726500006e74000069610000d3
:103fa0006c2000004d690000782000004f6e00007a
:103fb0002e0a00000d0000004c6500006674000031
:103fc0002053000074690000636b0000204400006f
:103fd0006966000066650000726500006e7400008e
:103fe000696100006c2000004d690000782000002d
:103ff0004f660000662e00000a0d0000005200000f
:1040000069670000687400002053000074690000b4
:10401000636b0000204400006966000066650000d4
:10402000726500006e740000696100006c20000081
:104030004d690000782000004f6e00002e0a00003d
:104040000d00000052690000676800007420000045
:1040500053740000696300006b2000004469000095
:104060006666000065720000656e000074690000fd
:10407000616c0000204d000069780000204f0000b6
:10408000666600002e0a00000d0000004d6500006d
:10409000636100006e7500006d2000005374000025
:1040a00065650000726900006e670000204d000029
:1040b00069780000204f0000666600002e0a0000ac
:1040c0000d0000004d650000636100006e7500008a
:1040d0006d200000537400006565000072690000e7
:1040e0006e670000204d000069780000204f00003e
:1040f0006e2e00000a0d0000004d000065630000f8
:10410000616e0000756d00002053000074650000b2
:1041100065720000696e0000672000004d690000b4
:10412000782000004f6e00002c2000007265000017
:104130006d61000070200000726900006768000077
:104140007420000073740000696300006b2000009d
:10415000792d000061780000697300002074000070
:104160006f2000000053000074690000636b0000c2
:10417000204800006f6c0000642f000052650000b2
:10418000636100006c6c0000206400006973000033
:10419000616200006c650000642e00000a0d0000e2
:1041a0000053000074690000636b000020480000a9
:1041b0006f6c0000642f0000526500006361000016
:1041c0006c6c000020740000696500006420000031
:1041d000746f0000204c00002d5300007469000033
:1041e000636b00002042000075740000746f0000d3
:1041f0006e2e00000a0d00000053000074690000dc
:10420000636b0000204800006f6c0000642f00000a
:1042100052650000636100006c6c000020740000b7
:104220006965000064200000746f000020520000e7
:104230002d53000074690000636b000020420000f1
:1042400075740000746f00006e2e00000a0d0000ef
:1042500000520000432000007365000072760000e9
:104260006f2000006d6f0000646500002e0a0000e2
:104270000d000000505700004d2000006d6f000041
:10428000646500002e0a00000d000000526100006d
:104290006e670000652000004f6600006673000036
:1042a00065740000203d0000200000005261000005
:1042b0006e670000652000003d2000000044000003
:1042c0006561000064620000616e0000642000000f
:1042d0003d20000000530000656e0000736900007f
:1042e000746900007669000074790000203d0000c8
:1042f00020000000486f00006d65000020500000a5
:104300006f73000069740000696f00006e20000088
:104310003d20000000430000616c00006962000065
:1043200072610000746900006e67000020410000a7
:104330006c6c0000204800006f6d000065200000dc
:10434000506f000073690000746900006f6e000018
:10435000732e00002e2e0000004f00007574000028
:104360007075000074200000496e00007665000042
:1043700072740000656400002e0a00000d00000049
:104380004f7500007470000075740000204e00002e
:104390006f7200006d6100006c2e00000a0d0000bd
:1043a000004f00007574000070750000742000005c
:1043b000546f0000676700006c6500002e0a000063
:1043c0000d0000004f75000074700000757400004f
:1043d00020530000696e0000676c0000652000003b
:1043e000536800006f7400002e0a00000d000000ea
:1043f0004f750000747000007574000020410000cb
:10440000757400006f66000069720000652e000080
:104410000a0d0000004f0000757400007075000068
:1044200074200000546f0000676700006c65000096
:1044300020410000757400006f6600006972000082
:10444000652e00000a0d0000004f0000757400008a
:104450007075000074200000507500007368000043
:1044600062750000747400006f6e00002e0a000078
:104470000d00000045520000524f00005220000085
:104480004f5500005450000055540000204d0000ce
:104490004f440000452e00000a0d000000500000af
:1044a000756c0000736500005769000064740000bb
:1044b000682000003d20000000300000206d00005a
:1044c000730a00000d00000041750000746f0000c9
:1044d00066690000726500002050000065720000ef
:1044e000696f0000642000003d20000000450000ce
:1044f000727200006f7200003a20000063610000d9
:1045000073650000206e00006f74000020680000da
:10451000616e0000646c0000656400002e0a0000fb
:104520000d0000002a2a00002a52000065730000d6
:1045300065740000204f0000757400007075000065
:10454000747300002e2a00002a2a00000a0d0000c1
:10455000004c00002d53000074690000636b0000e4
:10456000205800002d6100007869000073000000f1
:104570004c2d000053740000696300006b200000a4
:10458000592d00006178000069730000005200009e
:104590002d53000074690000636b00002058000078
:1045a0002d6100007869000073000000522d0000aa
:1045b00053740000696300006b200000592d000057
:1045c0006178000069730000004c00002d54000069
:1045d0007269000067200000616e0000616c0000dd
:1045e0006f670000005200002d5400007269000047
:1045f00067200000616e0000616c00006f670000c2
:10460000005800002d41000063630000656c00004d
:10461000657200006f6d0000657400006572000037
:10462000005900002d41000063630000656c00002c
:10463000657200006f6d0000657400006572000017
:10464000005a00002d41000063630000656c00000b
:10465000657200006f6d00006574000065720000f7
:10466000005a00002d470000797200006f730000af
:10467000636f00007065000000530000656c00006f
:10468000656300007420000062750000747400000f
:104690006f6e0000004c00002d5300007469000094
:1046a000636b00002062000075740000746f0000ee
:1046b0006e000000522d000053740000696300007a
:1046c0006b20000062750000747400006f6e0000c3
:1046d000005300007461000072740000206200004a
:1046e00075740000746f00006e000000442d00001f
:1046f000506100006420000055700000004400007c
:104700002d50000061640000205200006967000025
:1047100068740000004400002d5000006164000037
:10472000204400006f7700006e000000442d000060
:1047300050610000642000004c65000066740000b9
:10474000004c00002d54000072690000672000003a
:1047500062750000747400006f6e0000005200006b
:104760002d5400007269000067200000627500008f
:10477000747400006f6e0000004c00002d420000b9
:10478000756d00007065000072000000522d000081
:10479000427500006d70000065720000005400005a
:1047a00072690000616e0000676c00006520000007
:1047b00062750000747400006f6e0000004300001a
:1047c00069720000636c00006520000062750000e3
:1047d000747400006f6e000000430000726f0000f0
:1047e000737300002062000075740000746f000095
:1047f0006e000000537100007561000072650000da
:104800002062000075740000746f00006e000000ec
:10481000505300002062000075740000746f0000a7
:104820006e000000a9a20000b8a20000c7a200000c
:10483000d6a20000e5a20000f3a2000001a3000040
:1048400011a3000021a3000031a300003da300003c
:104850004ba300005aa3000069a3000076a3000048
:104860007fa300008ba3000096a30000a1a300007b
:10487000afa30000bda30000c6a30000cfa30000ab
:10488000dfa30000eda30000faa3000008a40000cd
:1048900045720000726f0000723a0000204900006b
:1048a0006e64000065780000206f000075740000e1
:1048b000206f000066200000726100006e6700003b
:1048c000652e0000200a00000d0000004368000073
:1048d000616e00006e6500006c20000000000000aa
:1048e000484f0000535400003a2000005553000088
:1048f00042200000424c000055450000544f00008b
:104900004f54000048200000494e00004954000068
:104910002e0d00000a000000474500004e3a00003e
:10492000205500005342000020470000656e000043
:104930006572000069630000204300006c6900009c
:10494000656e000074200000496e0000697400006c
:10495000616c0000697a0000656400003a20000084
:10496000666c000061670000733d00003078000055
:1049700000200000616400006472000065730000a4
:10498000733d00000020000056490000443d000037
:10499000307800000020000050490000443d000035
:1049a00030780000000d00000a000000484f0000b1
:1049b000535400003a2000005553000042200000ec
:1049c0005749000052450000204900004e490000b0
:1049d000542e00000d0a000000470000454e000064
:1049e0003a2000005553000042200000436f0000b1
:1049f0006e740000726f00006c6c00006572000045
:104a0000204300006c690000656e00007420000007
:104a1000496e000069740000616c0000697a000052
:104a2000656400003a200000666c000061670000c9
:104a3000733d000030780000005500005342000034
:104a400020470000656e0000657200006963000089
:104a5000204300006c690000656e000074200000b7
:104a60004465000076690000636500002044000092
:104a7000657400006163000068650000643a00002e
:104a80002061000064640000726500007373000020
:104a90003d00000053500000492000004275000016
:104aa000732000004d6f000064650000203000009e
:104ab0000a0d000000530000504900002042000091
:104ac00075730000204d00006f6400006520000039
:104ad000310a00000d000000535000004920000082
:104ae00042750000732000004d6f000064650000f7
:104af000203200000a0d0000005300005049000061
:104b00002042000075730000204d00006f6400001b
:104b100065200000330a00000d000000455200002f
:104b2000524f000052200000535000004920000066
:104b300042550000532000004d4f00004445000046
:104b40000a0d000000000000303100003233000088
:104b5000343500003637000038390000414200008b
:084b600043440000454600003b
:020000040000fa
:104b680062002000df4ce3000d003a0001407800ad
:104b78000c07070080007800420120000000e000d8
:104b880007003200204090000054a100a040980087
:104b9800214090000064a100a04098000001eb00b3
:104ba8000200780000000600eaccbf004600de00e4
:104bb8006100600000000600a066800001f020008f
:104bc800010060001203200016003200a066800079
:104bd80001f020000100600001402000810f50001a
:104be80007003a00a0668000000fb200a203200070
:104bf800f00f50000b0032000203200009003700bc
:104c0800a066800001f0200001006000220320005f
:104c180001502000810f500002003a00e0ccbf0094
:104c28000081fb000200780000000600e80ce200aa
:104c380007003a00200220005eee07004067880067
:104c48000000e000120032000008eb00010037000d
:104c5800220b070040678000906688008000eb0008
:104c6800a166880024adef008000fd00deecb700ef
:104c7800dfecb7008000fd00220da80040002000f6
:104c880060678800706788008167880010002000ce
:104c9800000006008f87e800889fbe008a9fbe003c
:104ca8008c9fbe008e1f7800014678000244780071
:104cb800830478000405be0006077800874678005c
:104cc80062002000df4ce30073003a00a066800019
:104cd80001f02000010060001200200001402000c7
:104ce800810f50006c003a0040678000304090000f
:104cf800020120000018a30067003200eb4f5400a7
:104d080025003a00326780000200e00052003200bd
:104d180053003700120178000200e0004e00320014
:104d2800624090000080fb00800f5500f9ff3a00b8
:104d3800220090000000e00047003200a000900030
:104d48000100e0004b003a000600370031409000b7
:104d58000018a30040003200910078000100e00034
:104d6800faff3a00920090000100e0003a00320099
:104d780044003700910078000100e000360032005e
:104d8800214090000080fb00808f5400f9ff3a001a
:104d98002101980008003700e14f540006003a004e
:104da8000300e00004003a00e24f560002003e0013
:104db800044078001f0d0700306680000c4878001a
:104dc80030668000184098003066800029409800be
:104dd800c848de00306680003140980030668000a8
:104de8004a409800c850de00306680005140980064
:104df800306680006b409800c858de00306680003e
:104e08007140980040678000afe8970011589800fb
:104e18000d04e00008003a00316680004067800019
:104e28000b0278008e01780082002000eb0a070050
:104e38000001eb00180037003166800040678000f1
:104e48000b0278008e01780082002000bf0a07005c
:104e58000001eb0010003700320020000e00370080
:104e6800624090000080fb00800f5200a9ff3a00ca
:104e7800afff3700314090000018a300b6ff3a009a
:104e8800f5ff3700214090000080fb00808f540020
:104e9800b8ff3a00beff3700020078004f077800dd
:104ea8004f06be004f05be004f04be002f00b100e4
:104eb80000000600889fbe008a1f780081417800a4
:104ec800020578000404be0062002000df4ce30005
:104ed80026003a00a066800001f020000100600072
:104ee8001200200001402000810f50001f003a00ee
:104ef800034078002b06070080017800420120005b
:104f08000000e00019003200500890000030b200a4
:104f18008201200015003200235890005201200021
:104f28000004e00011003d00234090001201200021
:104f38000058a3000d003a002340900022012000f1
:104f48000068a30009003a003340900002012000e5
:104f58000018a30005003200080178008a007800d4
:104f680003007800c90a07000001eb00020078007e
:104f78004f0578004f04be000000060061002000c5
:104f8800df4ce30008003a00a066800001f0200032
:104f98000100600031002000030032000000eb0037
:104fa800a0668800800078000100780000000600f4
:104fb80062002000df4ce30007003a00a166800091
:104fc8003200200000412000808f500002003a008b
:104fd800d42cec000001eb00020078000000060071
:104fe800881f78000144780062002000df4ce3004d
:104ff80013003a00a066800001f020000100600064
:105008001200200001402000810f50000c003a00df
:10501800460d0700220020000000e00008003a00ca
:1050280008007800dcecb70000c0eb0041678000a6
:105038009058980000332000a06688000001eb001b
:10504800020078004f04780000000600889fbe0028
:105058000204be0062002000df4ce3000e003a00ac
:1050680001407800cf050700800178004201200048
:105078000000e00008003200e1406400c508dd00df
:10508800304090000054a10001407000b0419800e9
:10509800891198000001eb00020078004f04be005f
:1050a800000006000200fa008000eb00412488009e
:1050b800dfccbf000b003200e1ff9f00240020007e
:1050c800050020000f81e900a106200094210700b7
:1050d800dfccbf0013002000f2cd20001107200014
:1050e800c80a07006000b800d0fe07000080fa0078
:1050f8000000060062002000df4ce30009003a00cf
:10510800a16680003200200000402000808f5000ff
:1051180004003a009404a90000412000a066880019
:105128000001eb0002007800000006000200fa000f
:10513800889fbe00f00ce2001f00320070678000fc
:1051480022cf2000e20f500003003c006c00b900a1
:10515800e2cf2000000141009200780020072000e3
:10516800808f500003003200f0ff2700808f50002e
:1051780004003a000281e800dfccbf00a300200051
:10518800a00a0700612480008c24ef00f02ced00b9
:1051980070678000e20f500003003c000000e80048
:1051a8007067880001003700ee2cef00612488004a
:1051b800f00ce200e1ff3a0020698000e10f4000b6
:1051c8000300320020698000a066880024adef004b
:1051d800a166800000f02000808060000020200090
:1051e800808f5000ba01320006003e000100e00046
:1051f8000e00320000102000808f50001b043a007f
:105208008b00370000402000808f5000bd03320023
:105218000010b000808f5000da0332000030200008
:10522800808f500011043a00ea013700a866800018
:10523800080fb200f00f5400560032000902200097
:10524800890f54005b0032000800e00007043a00b0
:1052580094ff0700406780000808780040678000d6
:105268001800980041678000314090000024a00099
:10527800b040980041678000314090000014a000c1
:10528800b0409800416780003140900009407000ac
:10529800b0409800017d2000406780000110980010
:1052a8000104200040678000410098006000b800b9
:1052b8004267800000099800110998004067800043
:1052c8002858980040678000085898004267800076
:1052d80052089000f1cf2f0001006000500998009b
:1052e80080c0eb00406780001158980030c0b300c0
:1052f800ceecb7000004fd00dcecb700ddecb70035
:10530800deecb7000004fd005867880038678800a5
:10531800b866880068248800f10f200051248800ae
:10532800c00820008224b6006f00500000248800c6
:10533800882488007124880000e020004800de00ee
:10534800c024880081002000a1248800a00020003b
:10535800a0248800a12488000003200030248800ad
:10536800200020003025880048258800b8248800bf
:10537800aae4a900a004200000258800a0668000f7
:1053880001ff20000100600070004000a066880056
:10539800b6033700220dab00b4033200a0668000cc
:1053a80001ff20000100600070004000a066880036
:1053b800ae0337008040eb00a1ff9f0020c3b3007d
:1053c800b0ff9f00240020000500200066815700e0
:1053d8009106200000c0eb00d12007000000e0008b
:1053e8000f00320010002000402488008ec0a90061
:1053f800f00f2f00ce20b60000602000ce20b700ae
:105408009ec0a800a066800001ff20000100600087
:1054180070004000a06688008cc4a8009303370081
:10542800220da90000012000a06688008f03370024
:10543800a1668000010fb20000022000808f50009a
:105448007b00320005003e000100e0000a00320047
:10545800f08f500085033a001d003700000320003c
:10546800808f5000d800320070004000808f5000bc
:105478007e033a000f013700a06680006f006000cd
:1054880003003200e20f500078033a000a003700a8
:1054980010002000502488008c04a800b00f2000c1
:1054a80080668800000420000024880082c4a800c8
:1054b800d42cec006d033700a066800001ff2000ab
:1054c8000100600070004000a06688006703370094
:1054d800a06680006f046000e20f540041003200b3
:1054e800e40f5400480032000800e0005f033a006f
:1054f800306680000000e00002003200bfec0700c8
:1055080038668800800020002aec07003066880092
:105518000000e00005003a0030c3b300e0ecb7003b
:1055280000502000a0668800500337000040eb00c0
:10553800dcecb700ddecb7000000eb00506788003a
:1055480031c0b3008000fd00cdecb7008000fd0045
:10555800d10020005125880060258800702588002a
:105568008025880090258800a0258800b02588001f
:10557800c0258800d0258800e0258800f02588000f
:1055880000268800102688002026880030268800fb
:10559800402688009444e20006003500ea0ca80082
:1055a80000c8b300deecb70000082000b024880073
:1055b800aae4a8009424a8009424a900ea8ca900cd
:1055c800eaaca9009484a800300320008066880013
:1055d8006d0040000024880082c4a800d42cec0090
:1055e800220337009484a9009404a800b000200086
:1055f80080668800000420000024880082c4a80077
:10560800d42cec0019033700f00020006024880037
:10561800f00f200080248800a066800001ff200091
:105628000100600070004000a06688000f0337008a
:10563800a06680006f006000e10f50002600320075
:1056480003003900e20f500008033a003600370023
:10565800806a80000000e0000200320067ec07006a
:10566800502def0001c8b300306680000148780073
:1056780061c0b30030668000114098000041eb0023
:10568800306680002240980011c0b3003066800068
:1056980031409800306680004240980030668000b3
:1056a8005240980081c0b300306680006140980085
:1056b8003066800072409800316680004067800044
:1056c8008400200081017800040178009f08070009
:1056d800d42cec00e502370041678000314090008f
:1056e8000018a300e1023200314090000008a30036
:1056f8000b0032003066800040409000e94f5000b7
:1057080005003a0050c3b300e0ecb7000050200099
:10571800a0668800d5023700d42cec00d3023700ed
:1057280058030700d1023700306680001080fb0064
:10573800a0eb070080007800806a88000000e00085
:1057480005003a0030c3b300e0ecb7000050200079
:10575800a0668800c502370030668000904878004f
:10576800704090000080fb0041678000c0009800f6
:105778003066800021ec0700c62cef0040678000ef
:10578800400090008beb0700306688000000e000c6
:1057980005003a0030c3b300e0ecb7000050200029
:1057a800a0668800b102370030c0b300cdecb70066
:1057b800a066800001ff200001006000700040002a
:1057c800a0668800a9023700a06680006f0060000c
:1057d800e10f50002400320003003900e20f5000ae
:1057e800a2023a002b003700d6ccbf0070416000ff
:1057f8009e023a0001c8b300306680000148780074
:1058080061c0b300306680001140980030668000a7
:105818002240980011c0b3003066800031409800e3
:105828003066800042409800306680005240980000
:10583800816a80003066800091407800614098005d
:105848003066800072409800836a8000316680006c
:10585800406780001382fb00820020003b0807009d
:10586800d42cec0081023700416780003140900061
:105878000018a3007d023200314090000008a30008
:1058880002003200d42cec0078023700fd02070039
:105898007602370030c0b300cdecb700a0668000b8
:1058a80001ff20000100600070004000a066880031
:1058b8006e02370050030700a066800001f0200048
:1058c800010060000010b000a06688006702370081
:1058d800a0668000000fb20064023a00a066800053
:1058e8006f006000e10f5000220032000300390011
:1058f800e20f50005d023a002900370010c0b300e3
:10590800dfecb7000041eb00306680000248780009
:1059180051c0b300306680001140980030668000a6
:10592800f1cd200091407800214098003066800039
:10593800324098003066800042409800306680000f
:1059480052409800306680006240980030668000bf
:105958007240980031668000406780000002eb00ca
:1059680084017800820020001c080700d42cec0079
:105978003e02370041678000314090000018a300c4
:105988003a023200314090000008a30002003200c1
:10599800d42cec0035023700ba0207003302370076
:1059a800eaccbf00610060004700dd00df4cb700b3
:1059b800deecb70030c0b300cdecb700a0668000c5
:1059c80001f02000010060000010b000a06688000f
:1059d80026023700a1668000010fb20000022000f5
:1059e800808f50008a00320005003e000100e00070
:1059f8000a003200f08f50001c023a001e003700e7
:105a080000032000808f5000cb003200700040005f
:105a1800808f500015023a0051013700806a8000db
:105a280010509000ccecb700206780000000e00028
:105a38000b00320010049000100078006feb070094
:105a4800206780000008eb00206780006beb0700f0
:105a580008007800286788000800e000f5ff3a0091
:105a6800a066800001ff2000010060007000400077
:105a7800a0668800fd013700a06680006f00600006
:105a8800e10f50002300320003003900e20f5000fc
:105a9800f6013a002a00370001c8b30030668000da
:105aa8000148780061c0b30030668000114098005a
:105ab800cc4ced0080407800306680002140980092
:105ac80021c0b30030668000314098000041eb00ef
:105ad800306680004240980030668000524098004e
:105ae80081c0b30030668000614098003066800055
:105af8007240980031668000406780008400200072
:105b0800810178000401780090070700d42cec008c
:105b1800d601370041678000314090000018a3008b
:105b2800d2013200314090000008a3000200320088
:105b3800d42cec00cd01370052020700cb0137000e
:105b4800600020009bea07000000e00005003a0022
:105b580030c3b300e0ecb70000502000a066880016
:105b6800c20137000004780031668000314090009f
:105b78004800dd00a14090008180fb00010040004a
:105b88008cea070000017800000c78000000e000b3
:105b980007003a000800780018eb070030c3b3008c
:105ba800e0ecb70000502000a0668800af01370085
:105bb80030668000b0409000c808dd0020409000aa
:105bc8000080fb008080400021419800c808de006a
:105bd80031419800216780001104980028678800e7
:105be80018017800726a8800ccccbf004044980045
:105bf80030c0b300cdecb700a066800001ff2000e4
:105c08000100600070004000a0668800970137001e
:105c1800a06680006f006000e10f50002d00320088
:105c280003003900e20f500090013a0034003700b9
:105c380001c8b300306680000148780061c0b30035
:105c48003066800011409800cc4ced008040780010
:105c5800306680002140980021c0b3003066800083
:105c6800314098008040eb00306680004140980049
:105c780030668000514098002067800090007800ce
:105c880030668000a1409000614098002067800045
:105c98009000780030668000b14090007140980014
:105ca8002067800090017800234190000281fb006a
:105cb800334290004822dd00316680004067800052
:105cc800020272008200200020070700d42cec009a
:105cd8006601370041678000314090000018a3003a
:105ce80062013200314090000008a3000200320037
:105cf800d42cec005d013700e20107005b0137009e
:105d080030c0b300cdecb700cc4ced00ccecb70004
:105d18000300320000312000a066880053013700dc
:105d2800a066800001ff20000100600070004000b4
:105d3800a06688004d013700a06680006f006000f3
:105d4800e10f50003f00320005003900e20f50001b
:105d580067003200e30f500044013a006f0037003b
:105d6800ac060700c2cd2000124178000204e00012
:105d780010003a0020678000506688000000e000ac
:105d88002200320010007800706a8800e8070700d7
:105d98000000e0001d003a009e06070050668000e3
:105da80010009000506688000000e00017003200e4
:105db800f4ff370021678000516688000100e00089
:105dc80026013a00090037005166880007003700ad
:105dd800910090000100e000fbff3200414090007c
:105de800804f5100faff3a00516688009100780010
:105df800716a8800ce070700000478000000e00000
:105e080002003a008306070058668800eaccbf0003
:105e18000028a30009003200ca0ce20005003a007d
:105e280040c3b300e0ecb70000502000a066880033
:105e38000e013700d42cec000c013700d42cec00f8
:105e48000a013700eaccbf00e440600022003a00b3
:105e5800ea4ca800306680000148780031c0b300e1
:105e68003066800011409800eaccbf000038a300db
:105e7800030032003066800021409800030037009c
:105e880041c0b30030668000214098008040eb009c
:105e980030668000314098003066800041409800ac
:105ea800306680005140980030668000614098005c
:105eb800306680007140980031668000406780003d
:105ec8000002eb008401780082002000c30607006e
:105ed800d42cec00e5003700a066800001ff20000c
:105ee8000100600070004000a0668800df003700f5
:105ef80041678000314090000018a300db003200a9
:105f0800314090000008a30002003200d42cec00bd
:105f1800d60037005b010700d400370030c0b3005b
:105f2800cdecb700ca0ce20005003a0040c3b3004c
:105f3800e0ecb70000502000a0668800cb003700d6
:105f480030c0b300cdecb700a066800001ff200090
:105f58000100600070004000a0668800c3003700a0
:105f6800a06680006f006000e10f50002200320040
:105f780005003900e20f50002a003200e30f5000fc
:105f8800ba003a002b0037000041eb003066800071
:105f98000248780091c0b300306680001140980034
:105fa80030668000c1cd20009140780021409800e3
:105fb8003066800032409800306680004240980089
:105fc8003066800052409800306680006240980039
:105fd800306680007240980031668000406780001b
:105fe8000002eb0084017800820020007b06070095
:105ff800d42cec009d0037004167800031409000b0
:106008000018a30099003200314090000008a30056
:1060180002003200d42cec0094003700190107006c
:106028009200370030c0b300cdecb700d42cec00a0
:106038008e003700a066800001f02000010060009b
:106048000010b000a0668800eaccbf000068a3007a
:106058001400320011ce20009140780001407800f1
:10606800a2c0b3000440bc008201780082c82000ae
:1060780002824100dfccbf00e302790034019000c6
:10608800c4019000050001000000e00077003a001c
:1060980090c3b300e0ecb70000502000a066880071
:1060a80072003700386780000800e0006f00320097
:1060b80089c82000f840900001407800a2c0b300d1
:1060c8000440bc0089014100dfccbf0062827c0033
:1060d80033019000c3019000040001000000e000bb
:1060e80004003a0090c3b300e0ecb7000050200071
:1060f800a0668800180478000800e0005b00320001
:10610800ecff3700a0668000000fb200f00f5000cf
:1061180056003a00a06680006f006000e30f500050
:106128000c003200e50f500013003200e10f500060
:106138004e003a009444a800500120008066880070
:10614800000420000024880082c4a800d42cec009d
:10615800460037009444a9009404a800b000200029
:1061680080668800000420000024880082c4a800fb
:10617800d42cec003d00370000402000a0668800c9
:106188003a003700a2668000020fb20037003a00da
:1061980080002000a024880062248800f10f2000dd
:1061a80051248800c00820008224b6006f005000e7
:1061b8000024880082248800712488008c04a800a8
:1061c80002ce20001241780040c3b300c1c6b3001c
:1061d800804f51001500320007003e008140e80062
:1061e800e74f5100110032000040e900804f510094
:1061f8000b003a000800370051c6b30050c3b30083
:10620800804f51000900320064404000804f510027
:1062180003003a0004003700f1c6b300030037005a
:1062280001c7b30001003700e1c6b3008180fb005d
:10623800dfccbf00140020000500200022ce200083
:10624800371d0700a066800001ff200001006000e4
:1062580070004000a06688000400370041409000ac
:10626800804f5100dafe3a00e0fe37004f04be00ce
:106278000080fa0000000600df4ce3000b003a0043
:106288000140780047010700800078000000e00026
:1062980006003200204090000074a000a040980042
:1062a800314090000014a000b040980000000600a3
:1062b800889fbe000204be00df4ce30006003200e7
:1062c80060c0b300004978008009eb00b311780082
:1062d800100020002300370001407800310107003a
:1062e800800078000000e0001b0032003040900081
:1062f8000000d10061416000314090000008a30017
:1063080005003200004ceb00010a9000910a900051
:10631800848cbe000e003700214090000058a30076
:106328000300320010c1b300004c780008003700a9
:10633800214090000068a30003003200c15890007b
:10634800014c78000200370090c1b300004c78007f
:106358000280fb000300370040c1b300004c780006
:10636800100020004f04be000000060080017800e5
:10637800e1cf40000f003a000204e0000d003a00af
:1063880080062000808f510004003a0045fb07007a
:10639800220da9000000eb0007003700b00620001e
:1063a800808f510003003a00220da8000000eb0086
:1063b800010037003000200000000600889fbe0062
:1063c8008a1f780081417800020578000404be0025
:1063d80062002000df4ce30026003a00a06680003f
:1063e80001f02000010060001200200001402000a0
:1063f800810f50001f003a0003407800e9000700b1
:1064080080017800420120000000e00019003200fd
:10641800500890000030b2008201200015003200c0
:1064280023589000520120000004e00011003500bc
:1064380023409000120120000058a3000d003a00ec
:1064480023409000220120000068a30009003a00c0
:1064580033409000020120000018a300050032001c
:10646800080178008a00780003007800b605070064
:106478000001eb00020078004f0578004f04be00d1
:106488000000060091668000214090000064a10091
:10649800a040980091668000214090000054a1001f
:1064a800a0409800cd4ced00cdecb70003003200c1
:1064b80000ff2f00d42cb6000a003700ce4ced00a8
:1064c800ceecb7000300320000112000a06688005f
:1064d8000400370070c0b300e0ecb70000502000a3
:1064e800a066880000000600ee874700889fbe006f
:1064f8008a9fbe008c9fbe008e1f78008046780061
:1065080001477800e2ef9f0083bf9f008b6a8000fd
:106518000004eb00e9c92000ccc920004345dd0098
:106528006600450060007e000018a30027003200c6
:1065380069f897008d4f500024003a0079f89700c9
:106548008e4f500021003a006fe89700994f1000d5
:106558001e003a008b4890008180fb001b48900089
:106568004800dd0081007000b1b79f00ab48900083
:106578008180fb003b4890004800dd00010070006e
:10658800c0b79f00adef9f00beef9f00efe89700f8
:10659800c1ef9f0084002000050020007a81570089
:1065a8009107200000c0eb005d1c07000000e00020
:1065b80006003a000a004600504090008fb8970045
:1065c8008048780010002000050037000804e80023
:1065d800e8844400e20f5400d0ff3a000000eb00ca
:1065e8004f0778004f06be004f05be004f04be009f
:1065f800ef00b100000006000800fa00889fbe0006
:106608008a9fbe008c1f7800886a8000eacca900a7
:106618000005eb00e9c92000cbc920000b06780073
:106628004350dd006600400060007e000018a300b3
:106638000c003200484090009b4f100039003a008f
:10664800f9f897005840900080cf500035003a0084
:1066580068409000994f100032003a00eacca80038
:10666800300037009b017800884890008180fb004b
:10667800184890004800dd0001007000808f51002c
:1066880008003a00a84890008180fb003848900034
:106698004800dd0001007000990f100001003a0069
:1066a800eacca800e18f41001e003a000080eb0010
:1066b800990f10001b003a00884890008180fb0069
:1066c800184890004800dd0081007000f1b79f0075
:1066d800a84890008180fb00384890004800dd0001
:1066e8000100700080bf9f001b407800a0f79f004a
:1066f80079f89700b0f79f0019407800c0f79f001d
:1067080084002000050020007281570091072000b6
:1067180003407800021c07000000e00001003a0076
:10672800eacca800eaccbf000068a3001100320040
:106738004351dd008200460051409000e1ecb70073
:106748006600410060007e00110020000028a300c0
:106758000e0032004350dd0064004000801f7800c6
:1067680060407e00dcecb7004f007800110020008c
:10677800060037000a05e800e8844400e88545007b
:10678800e20f5500a6ff3a008000eb0001007800f8
:106798004f0678004f05be004f04be000080fa0087
:1067a80000000600004178000004e00002003a0002
:1067b8004167800018003700336780000300e0005d
:1067c80010003200230090000000e0000a003200b0
:1067d800a00090000100e0000c003a00060037001d
:1067e80021589000804f51000b0032009100780032
:1067f8000100e000faff3a00930178000300e0008e
:10680800f0ff3a008000eb000300370021589000a9
:10681800804f5100f5ff3a000100780000000600a3
:10682800889fbe008a9fbe00a0668000d6ccbf00ad
:106838000048a30099033a00d6ccbf008005eb00be
:106848000008a300af013a000040eb0096030700e0
:106858000000e00002003a0080057800a801370037
:10686800926680000258900080007800010fb20004
:1068780000022000808f5000880032007000400025
:10688800808f500012013200f08f50007b033a00d5
:10689800025890006f006000e10f500014003200b1
:1068a80003003c000000e0000600320073033700dc
:1068b800e20f50001e003200ef0f50006f033a0045
:1068c80049003700324090000034a1003041980060
:1068d800d0c0b3009506070090668000205890004d
:1068e800d1c0b30074060700d60ca8006b033700ac
:1068f80002089000920890005001980061019800e9
:1069080091668000314090000034a000b0409800ab
:1069180090c0b3008506070090668000205890005c
:1069280091c0b30064060700d60ca8005b033700cb
:106938000040eb00005998009166800031409000bb
:106948000014a000b040980080678000e30f50005a
:1069580020003c000000e800806788006067800035
:10696800e20f500003003c000000e8006067880068
:1069780001003700ec2cef00606780006c00b90064
:1069880022cf2000000141002007200000097800e4
:1069980091668000010a9000910a90001401980005
:1069a80025019800b10a9000350198000040eb00dd
:1069b800104998002158900000499800b15990005a
:1069c8002349980091589000314998008005eb00c0
:1069d8004b01370081c0b3009066800031589800a1
:1069e8008005eb00460137000040eb000059980095
:1069f80091668000314090000014a000b0409800db
:106a080080678000e30f50001f003c000000e80092
:106a18008067880060678000e20f500003003c0038
:106a28000000e8006067880001003700ec2cef00e8
:106a3800606780006c00b90022cf2000000141008f
:106a4800f0ff2700000978006000b80010019800e6
:106a5800210198008000eb003101980090668000c9
:106a6800405a900014499800a05a9000054998008f
:106a7800b059900023499800105890003049980068
:106a8800810578001e01370081c0b3009066800040
:106a9800315898008005eb00190137000258900022
:106aa8006f006000e20f50001e00320005003c003d
:106ab8000000e00008003200e10f5000ef023a0049
:106ac80010003700e30f500026003200ef0f50008f
:106ad800ea023a0051003700324090000034a10029
:106ae80030419800d0c0b3001006070090668000bf
:106af80020589000d1c0b300ef050700d60ca800bd
:106b0800e602370090c0b3000806070090668000d0
:106b18002058900091c0b300e7050700d60ca800e4
:106b2800de023700020a9000920a90005401980091
:106b38006501980091668000314090000034a00003
:106b4800b040980010c0b300f805070090668000b8
:106b58002058900011c0b300d7050700d60ca80034
:106b6800ce0237000040eb00005998009166800083
:106b7800314090000014a000b04098008067800069
:106b8800e30f500020003c000000e8008067880008
:106b980060678000e20f500003003c000000e8003e
:106ba8006067880001003700ec2cef006067800008
:106bb8006c00b90022cf200000014100200720000e
:106bc8000009780091668000010a9000910a9000ff
:106bd8001401980025019800b10a90003501980029
:106be8000040eb0010499800215890000049980097
:106bf800b159900023499800915890003149980064
:106c08008005eb00be00370081c0b30090668000ad
:106c1800315898008005eb00b90037000040eb00c0
:106c28000059980091668000314090000014a0003f
:106c3800b040980080678000e30f50001f003c00c0
:106c48000000e8008067880060678000e20f50005d
:106c580003003c000000e80060678800010037007e
:106c6800ec2cef00606780006c00b90022cf200098
:106c780000014100f0ff2700000978006000b8001b
:106c880010019800210198008000eb003101980064
:106c980090668000405a900014499800a05a9000cd
:106ca80005499800b0599000234998001058900061
:106cb80030499800810578009100370081c0b30001
:106cc80090668000315898008005eb008c003700f2
:106cd800025890006f006000e20f50001e00320062
:106ce80005003c000000e00008003200e10f500001
:106cf80062023a0010003700e30f5000260032000d
:106d0800ef0f50005d023a0051003700324090000a
:106d18000034a10030419800d0c0b30083050700bb
:106d28009066800020589000d1c0b300620507002b
:106d3800d60ca8005902370010c0b3007b05070025
:106d4800906680002058900011c0b3005a050700d3
:106d5800d60ca80051023700020a9000920a90004f
:106d680054019800650198009166800031409000b8
:106d78000034a000b040980090c0b3006b05070035
:106d8800906680002058900091c0b3004a05070023
:106d9800d60ca800410237000040eb0000599800cb
:106da80091668000314090000014a000b040980027
:106db80080678000e30f500020003c000000e800de
:106dc8008067880060678000e20f500003003c0085
:106dd8000000e8006067880001003700ec2cef0035
:106de800606780006c00b90022cf200000014100dc
:106df800200720000009780091668000010a9000b1
:106e0800910a90001401980025019800b10a900099
:106e1800350198000040eb00104998002158900077
:106e280000499800b1599000234998009158900062
:106e3800314998008005eb003100370081c0b3006c
:106e480090668000315898008005eb002c003700d0
:106e58000040eb0000599800916680003140900096
:106e68000014a000b040980080678000e30f500035
:106e78001f003c000000e800806788006067800011
:106e8800e20f500003003c000000e8006067880043
:106e980001003700ec2cef00606780006c00b9003f
:106ea80022cf200000014100f0ff270000097800f0
:106eb8006000b80010019800210198008000eb00e4
:106ec8003101980090668000405a9000144998005b
:106ed800a05a900005499800b0599000234998009d
:106ee8001058900030499800810578000400370058
:106ef80081c0b30090668000315898008005eb008f
:106f0800d60ca800d6ccbf000018a300f1003200b0
:106f1800f5003700926680000258900080007800e3
:106f2800010fb20000042000808f500004003200de
:106f380070004000808f5000db003a006c00370082
:106f4800025890006f006000e10f50000b00320003
:106f5800ef0f5000380032000000e000d2003a0085
:106f680090c0b300f104070090668000205890009c
:106f780091c0b300d0040700c80137000040eb00ff
:106f88000059980090668000200290003400980014
:106f980091668000314090000014a000b040980035
:106fa80080678000e30f50001f003c000000e800ed
:106fb8008067880060678000e20f500003003c0093
:106fc8000000e8006067880001003700ec2cef0043
:106fd800606780006c00b90022cf200000014100ea
:106fe800200720000009780091668000010a9000bf
:106ff800910a90001401980025019800b10a9000a8
:10700800350198000040eb00104998002158900085
:1070180000499800b1599000234998009158900070
:10702800314998009d00370081c0b3009066800008
:1070380031589800990037000040eb00005998003b
:1070480090668000200290003400980091668000cd
:10705800314090000014a000b04098008067800084
:10706800e30f50001e003c000000e8008067880025
:1070780060678000e20f500003003c000000e80059
:107088006067880001003700ec2cef006067800023
:107098006c00b90022cf200000014100f0ff27005a
:1070a800000978006000b8001001980021019800dc
:1070b8000000eb003001980090668000c05a9000f4
:1070c80015499800a058900001499800b0599000bf
:1070d8002349980010589000304998006f003700f5
:1070e80081c0b30090668000315898006b0037006b
:1070f800025890006f006000e10f50000b00320052
:10710800ef0f5000380032000000e00066003a003f
:1071180010c0b300850407009066800020589000d6
:1071280011c0b300640407005c0137000040eb00a5
:107138000059980090668000200290003400980062
:1071480091668000314090000014a000b040980083
:1071580080678000e30f50001f003c000000e8003b
:107168008067880060678000e20f500003003c00e1
:107178000000e8006067880001003700ec2cef0091
:10718800606780006c00b90022cf20000001410038
:10719800200720000009780091668000010a90000d
:1071a800910a90001401980025019800b10a9000f6
:1071b800350198000040eb001049980021589000d4
:1071c80000499800b15990002349980091589000bf
:1071d800314998003100370081c0b30090668000c3
:1071e800315898002d0037000040eb0000599800f6
:1071f800906680002002900034009800916680001c
:10720800314090000014a000b040980080678000d2
:10721800e30f50001e003c000000e8008067880073
:1072280060678000e20f500003003c000000e800a7
:107238006067880001003700ec2cef006067800071
:107248006c00b90022cf200000014100f0ff2700a8
:10725800000978006000b80010019800210198002a
:107268000000eb003001980090668000c05a900042
:1072780015499800a058900001499800b05990000d
:1072880023499800105890003049980003003700af
:1072980081c0b30090668000315898000b00e00070
:1072a80002003a000b0037001b0020008040eb0072
:1072b8009066800001589800906680002002900037
:1072c8003400980091668000314090000014a000be
:1072d800b040980030c0b300f30007000000e000a1
:1072e8000cff3a00d62ca800d6ccbf000038a3006b
:1072f800ea003a000044eb0029cf20008ac0b3001e
:1073080020c0b300e80007000000e000d20032000f
:10731800926680000258900080007800010fb20049
:1073280000082000808f50000400320070004000e8
:10733800808f5000c1003a005f003700025890006b
:107348006f006000e10f50000b003200ef0f50009b
:10735800310032000000e000b8003a0090c0b300ed
:10736800f2030700906680002058900091c0b30097
:10737800d1030700c90037000859980091668000ba
:10738800314090000014a000b04098008067800051
:10739800e30f50001d003c000000e80080678800f3
:1073a80060678000e20f500003003c000000e80026
:1073b8006067880001003700ec2cef0060678000f0
:1073c8006c00b90000804400220720000208780001
:1073d80092668000020a9000920a900014009800b9
:1073e80025009800b20a90003500980018489800c7
:1073f800a258900001489800b2599000234898007c
:107408001259900032489800890037009066800031
:107418003a5898008600370008599800916680000d
:10742800314090000014a000b040980080678000b0
:10743800e30f50001d003c000000e8008067880052
:1074480060678000e20f500003003c000000e80085
:107458006067880001003700ec2cef00606780004f
:107468006c00b90000804400f2ff27000208780091
:107478006011b80012009800230098000001eb008a
:107488003200980092668000425a90001448980092
:10749800a25a900005489800b258900021489800d8
:1074a80012599000324898006100370090668000b9
:1074b8003a5898005e003700025890006f0060004c
:1074c800e10f50000b003200ef0f50003100320086
:1074d8000000e00059003a0010c0b3009303070011
:1074e800906680002058900011c0b3007203070016
:1074f8006a00370008599800916680003140900072
:107508000014a000b040980080678000e30f50008e
:107518001d003c000000e80080678800606780006c
:10752800e20f500003003c000000e800606788009c
:1075380001003700ec2cef00606780006c00b90098
:10754800008044002207200002087800926680002c
:10755800020a9000920a90001400980025009800f2
:10756800b20a90003500980018489800a258900078
:1075780001489800b2599000234898001259900089
:10758800324898002a003700906680003a589800e0
:107598002700370008599800916680003140900014
:1075a8000014a000b040980080678000e30f5000ee
:1075b8001d003c000000e8008067880060678000cc
:1075c800e20f500003003c000000e80060678800fc
:1075d80001003700ec2cef00606780006c00b900f8
:1075e80000804400f2ff2700020878006011b8000c
:1075f80012009800230098000001eb003200980068
:1076080092668000425a900014489800a25a90004e
:1076180005489800b25890002148980012599000e7
:107628003248980002003700906680003a58980067
:107638000b00e00002003a00070037001b002000a2
:10764800906680000858980091668000314090004c
:107658000014a000b0409800d94ce20005003200a8
:10766800d86cef00d6ccbf000038a3000b003a005e
:1076780023ff3700d66ca800080037000040eb0055
:107688000059980091668000314090000014a000d5
:10769800b04098001b00200019fe37004f05be00bf
:1076a8004f04be00000006000042780041678000d9
:1076b8008082fb00510890004800de0063006000f3
:1076c800850f500006003a00314090000018a300d2
:1076d80003003a0091668800100020004c00370033
:1076e800d96cef00336780000300e00047003200e8
:1076f800230090000000e00007003a000001780035
:107708003f003700d9ccbf00d8ecb700926688009c
:10771800100020003e00370020019000380037009c
:10772800520890004800de0063006000808f52001d
:1077380027003a00e24f520019003200e34f52008e
:10774800080032000404e00021003a0032409000b2
:107758000018a3001e003a0092668800100020005e
:107768002b003700324090000018a30006003200ba
:10777800320090000000e00015003a00220090005e
:107788003001980012003700320090000000e0003d
:107798000f003a0092668800100020001c00370095
:1077a800324090000018a30009003a0032409000cf
:1077b8000048a30006003a00d96cec0091cd2000e7
:1077c80091407800d8ccbf0080cf5000cdff3e005c
:1077d800120178000200e00009003a0093017800e5
:1077e8000300e00009003200230090000000e000e0
:1077f80002003a00000178000100370020019000e3
:107808000200e000c6ff3a00f4ff37000000eb007a
:1078180000000600889fbe008a9fbe003b6780006c
:107828000b00e000280032009b05780030678000dc
:10783800900090000100e0001f0032001105780060
:107848003067800090009000210090000000e00068
:107858000e0032008004eb0010047800e7e3070014
:107868003067800010009000290098003067800081
:107878001000900028009800306780009000900069
:10788800210090000000e000f3ff3a0001007800ba
:10789800dae307000000eb003167800090009800f1
:1078a800306780001a0098003067800090009000d0
:1078b8000100e000e1ff3a00d0e307003b678800e1
:1078c8000b00e000d8ff3a0040678000906688000f
:1078d8004f05be004f04be0000000600881f780058
:1078e800206780000000e0000b00320010049000c8
:1078f80010007800c1e30700206780000008eb0053
:1079080020678000bde3070008007800286788002a
:107918000800e000f5ff3a00806a80000000e000ff
:1079280002003200b5e30700502def0030668000fa
:107938000000e00002003200b0e30700c62cef00b0
:10794800b4ff07004f04780000000600a042900032
:107958000554a10025409800a04290000564a100ac
:1079680025409800a04290000574a1002540980089
:10797800b04290000504a10035409800a042900054
:1079880006ceb30086c2620025409800b04290003f
:107998000544a10035409800330898006033b800ca
:1079a8000608980017089800050020005400980061
:1079b800650098008001eb00730898002108980082
:1079c8007200980001c2b30001589800b0409000be
:1079d8000114a1003140980000000600881f7800bb
:1079e80000047800204090000054a1002044980032
:1079f800284090000064a10020449800284090008e
:107a08000074a10020449800384090000004a100b0
:107a1800304498002840900005ceb300054060002f
:107a280020449800384090000044a1003044980059
:107a3800330c98006033b800060c9800170c9800b7
:107a48006123b80056049800670498000000eb0012
:107a5800700c9800210c9800720498000400e00053
:107a680003003a0000c1b300005c98000200370030
:107a780000c3b300005c9800384090000014a100d7
:107a8800304498004f047800000006008001780018
:107a980002027800204090000074a100a0419800e4
:107aa800334090000004a100b041980023409000aa
:107ab80002ceb30002406000a0419800334090001d
:107ac8000044a100b0419800b10998006000b800d6
:107ad80080099800910998006120b800d0019800a9
:107ae800e10198000000eb00f0099800d30890002d
:107af8000030200080806000808f500003003a0032
:107b080000c4b300805998000b0037000010200013
:107b1800808f500006003a0000c6b30080599800d4
:107b2800b30890000040eb00904098000200370036
:107b380000c8b30080599800334090000014a10099
:107b4800b041980000000600800178000202780029
:107b5800204090000074a100a0419800334090009c
:107b68000004a100b04198002340900002ceb30069
:107b780002406000a0419800334090000044a100fa
:107b8800b0419800b10998006000b80080099800d9
:107b9800910998006120b800d0019800e10198008f
:107ba8000000eb00f0099800d30890000030200096
:107bb80080806000808f500003003a0000c5b30049
:107bc800805998000b00370000102000808f50006b
:107bd80006003a0000c7b30080599800b308900027
:107be8000040eb00904098000200370000c9b30045
:107bf80080599800334090000014a100b0419800cb
:107c080000000600889fbe008a9fbe008c9fbe00b1
:107c180080467800810478000205be002007200015
:107c2800808f500003003200f0ff2700808f500043
:107c38000e003a001a489000e14f40001c00320044
:107c4800a2c0b3000440bc000281e80080c8200044
:107c5800e2017800615ab8000a01780089007800ca
:107c68000d407800030001001100370038678000dc
:107c78000800e0000e0032008cc820007840900018
:107c8800a2c0b3000440bc000281e800e2017e000b
:107c9800615ab8000a017800890078000d40780020
:107ca80003000100180478000800e000f3ff3a0020
:107cb8004f06be004f05be004f04be000000060080
:107cc800889fbe008a9fbe008c9fbe000046780039
:107cd8008105780002057800830478003867800001
:107ce8000800e0000e0032008dc8200078409000a7
:107cf800a2c0b3000440bc0064014100e2817e00e0
:107d0800614ab8000a0178008b0078000c407800be
:107d180003000100180478000800e000f3ff3a00af
:107d28004f06be004f05be004f04be00000006000f
:107d3800ec874700889fbe008a9fbe008c9fbe00cc
:107d48008e1f7800726a800039678000ea2ca900cb
:107d5800ea4ca80012447800a24090008180fb0001
:107d6800324090004800dd000087400052409000fb
:107d7800e0ef9f0002499000f2ef9f0077815700e3
:107d8800ffe89700114198000049eb00240020000b
:107d9800050020009106200000c0eb0060160700d7
:107da8000002eb000000e00003003a0080c2b300cc
:107db800e0ecb700140020008880fb00706a8000a7
:107dc800008440000400e000ce003a0081057800fd
:107dd800d4ef9f00c500370014002000c900370009
:107de80018467800984090000880e800e9cf5000d5
:107df8000c003a00ea2ca80010407800ddecb7002f
:107e08000018a30005003200eaccbf000038a30028
:107e180002003200ea4ca90004003700ea6ca9000d
:107e280002003700e4cf5000050032000c80fb0050
:107e380080854500706a800000844500ae003700e8
:107e480090467800b840900091f79f004840900015
:107e580080f79f0058429000e840900078419000d9
:107e680068044400eaccbf000068a30003003200a5
:107e7800e1ccbf0080ef9f000a003700f88157006f
:107e88000440780098f907000000e00005003a0077
:107e98000c80fb0080854500706a800000844500e6
:107ea800950037000900e000cb003a0008003700d1
:107eb800090578001a0578000a00e000040032007d
:107ec8006a40900080cf560010003200f9ff37005a
:107ed80080002000b7e10700000578000000e000fe
:107ee800750032006d4098008fe897007140980047
:107ef8000000eb001005980020059800090d780097
:107f08008a04780001003700090578006000200025
:107f1800a8e10700800678000000e000a1003a0010
:107f2800650037002d0598000c80fb008085450012
:107f3800706a8000008445000040eb00c0ef9f009d
:107f4800a2003700184678000885e800184090001d
:107f5800e54f500009003200dfe89700c1ef9f00ad
:107f68000c80fb0080854500706a80000084450015
:107f7800960037004fe89700d0ef9f0020022000be
:107f88008ce10700800178000000ea00030070001f
:107f9800cf02de0010c0b300854250000582fb000e
:107fa8001a457800aa599800b8409000b15998002d
:107fb800c84090008180fb00c101980058409000a3
:107fc8004800dd0080804000c101980068409000b2
:107fd8000083fb00a60198000001eb0092019800c5
:107fe800334090000024a000b04198003340900036
:107ff8000014a000b04198006000b8008009980003
:1080080091099800825998000fe8970090599800b4
:10801800530890000030b20001102000810f50007a
:1080280011003a000600e00002003a0010002000ab
:10803800a001980023009000f00f500002003600c5
:1080480000012000a0019800230090000000e90032
:10805800110020008008dd00a10198003340900045
:108068000024a100b0419800a3009000b10198003d
:108078002d00900080097800a3069800dfe897009b
:108088008140e800d1ef9f000c80fb00808545000f
:10809800706a8000008445000504e0000d003a0085
:1080a8008b0f5700060036000ff0970080cf500066
:1080b800a4ff3a0002003700140020000500370032
:1080c8000002eb0003003700cfe89700d1ef9f00d4
:1080d8000002eb005fe897008ff09700814f500097
:1080e8003dff3a000400e00006003a008b0f5700fd
:1080f8003bff3e00030037008b0f570038ff3e0060
:108108000002eb000900e000410032000400e0003a
:108118001a00320019057800190490000800e000e0
:108128001000320018007800900498002800900091
:108138000000e0000600320090007800210498005a
:10814800aee10700280090000000e000faff3a00c6
:1081580008007800a9e10700190490000800e00071
:10816800f0ff3a0009007800a4e107000a00e000e7
:108178000a0032008a047800e6ff37006fe89700ab
:10818800dcecb700ffe897000180fb00106788006f
:108198003967880010002000200037000000eb003d
:1081a8001e0037001a009000800e78009ff097009c
:1081b800a14698000000eb00a00698001d05980055
:1081c8000104e00057ff320057ff37008b0f5700bc
:1081d80005003e00bcff37006940900080cf560084
:1081e80033ff3a0048ff37004fe897008ff09700b9
:1081f800814f5000b4ff3100184678000885e80028
:1082080018409000e54f500055ff3a0059ff3700dd
:108218000900e000bfff3a00e0ff37004f07780091
:108228004f06be004f05be004f04be00cf00b10090
:10823800000006000004e00017003a0034678000e0
:108248000400e0001b003200940190000300e000ed
:108258000d003200a30090000100e000070032008a
:1082680072cfb3003140900002406000b0409800e7
:10827800910078000100e000faff3a0093017800cd
:108288000300e000f3ff3a00140278000400e00065
:1082980008003200ecff370042f907008000780040
:1082a8000000e00003003200304090000034a100dc
:1082b800b04098000000060000427800eaccbf00f9
:1082c800d3cdb3000008a30001003a00d3c5b30022
:1082d80092668000325890006340600001003a00c6
:1082e8000344a1003258900063406000e14f500001
:1082f80001003a000304a1000380fb005025880018
:10830800deccbf000080fb00b02488000180fb00a9
:108318004400dd0084007800f107b200010070001d
:10832800f0248800d68ca8000000060000417800e0
:10833800e94f500011003a00eaccbf0047e02000a6
:108348000048a30001003a0007e02000eaccbf0083
:108358004400de00610060000004a2004400dd006b
:10836800a1ce2000914078000144a10080c0700097
:1083780001007800eaecb70025003700eaccbf001e
:10838800c7e020000058a30001003a0087e0200061
:10839800eaccbf004500de00610060000004a200d6
:1083a8004500dd00a1ce2000914078000154a100d5
:1083b80080c0700001007800eaecb700ed4f510072
:1083c80013003a009666800076009000060a900036
:1083d800960a900046019000010020000400500019
:1083e8008580580003002000820f5000838f5800ba
:1083f80002003600c60190001f0037007601900089
:108408000608900096089000800151001a00370075
:10841800966680003658900063406000e14f500037
:1084280002003a00c60190003b0037005600900059
:10843800e6009000060a9000960a90004601900017
:10844800040050008580580003002000820f50006f
:10845800838f580002003600c60190002e003700b6
:1084680056019000e60190000608900096089000da
:108478008001510028003700260b900096039800d1
:108488000e003700b60890003608900010409000a3
:1084980062c0b3000440bc0066014100e28078007d
:1084a80091039800050037003609900006089000ef
:1084b8009608900000014100920398000040eb00ec
:1084c8009043980083007800f13fb20000c02f006d
:1084d800970b6000978b7000916680003140900088
:1084e8004300de00610060004e00dd0017e0a100df
:1084f800970b7000314090004200de006100600080
:108508004b00dd0017b0a100970b70000000280099
:10851800970b70000000060036589000634060001a
:10852800e14f5000e0ff3a00d6ff37004067800077
:10853800304090000018a300170032003367800015
:108548000300e00016003200130190000200e00072
:108558000d003200a20090000100e00012003a0075
:1085680006003700314090000018a3000a003200ce
:10857800910078000100e000faff3a00120178004b
:108588000200e000f3ff3a00930178000300e000e6
:1085980003003200ecff370010002000060037000f
:1085a8000000eb0004003700314090000018a300e1
:1085b800efff3a00f8ff3700000006003600f80029
:1085c800809fbe00829fbe00849fbe00869fbe0023
:1085d8008ec0a90082c4bf000068a300100032004a
:1085e80080c4bf000068a3000d0032000004200012
:1085f80000248800d00ce20009003200d02ced00e5
:10860800d00ce20006003a0082c4a900a0668000ef
:1086180001f020000100600001003200d42cec00c1
:108628008cc4bf000068a3000c0032008ac4bf00dd
:108638000068a300090032008cc4a90000042000cf
:1086480050248800a166800070005000808f500080
:1086580002003a0000102000206988008cc4bf0086
:108668000008a300070032008ac4bf000008a30066
:108678000400320010002000502488008c04a90057
:10868800242def008cc4bf000038a300370132004e
:108698008ac4bf000038a300340132008cc4bf0074
:1086a8000018a300080032008ac4bf000018a30005
:1086b80005003200906680003058900063406000ea
:1086c800e14f500029013a00d68ca900922480007d
:1086d800800020005024880093668000a3589000f2
:1086e800f0248000ef8060006f006000808f5000f1
:1086f8001d013a00020078000238a300050032008c
:10870800c2e020000028a30006003a0082e0200012
:108718000400370042e020000028a30001003a00ce
:1087280002e0200000c023009200600000802000ca
:10873800808f500046003a00f03f2000920260000f
:10874800030890009308900005004000e08048006e
:1087580080099800910998008000eb0090668000dd
:108768007108980092668000324090004300de0055
:10877800610060000004a2004300dd00b2409000e8
:108788000134a10080c070003141980094668000d7
:1087980004589000f04f50000800320084589000b0
:1087a80000c2b30080cf500004003200845890000b
:1087b8007040400080cf50000f003a00040990003c
:1087c800940990007400900001002000800f51006f
:1087d800818f5900e40039006000b800000a980051
:1087e800110a980091668000015890000040e80046
:1087f80080589800dc0037003458900063406000cf
:10880800e14f50000a00320044009000808f52006f
:108818000700390004099000940990005400900062
:10882800e4009000800f5100818f5900ce0039007c
:10883800344090000004a000304298009166800007
:10884800015890000040e80080589800c6003700a2
:1088580000c02000808f50000300320000c02200ba
:10886800808f50002c003a00f03f200092026000f8
:10887800030890009308900005004000e08048003d
:1088880080099800910998008000eb0090668000ac
:108898007108980092668000324090004300de0024
:1088a800610060000004a2004300dd00b2409000b7
:1088b8000134a10080c070003141980094668000a6
:1088c8003458900063406000e14f50000a003200c5
:1088d80044009000808f520007003900040990007e
:1088e8009409900054009000e4009000800f51001b
:1088f800818f59009c003900344090000004a0008a
:108908003042980091668000015890000040e800cd
:10891800805898009400370000802200808f500013
:1089280064003a00334090000044a000b041980031
:1089380091668000710890000000e800f008980037
:10894800926680003258900063006000e10f50008a
:108958005000320003003c000000e0001a00320022
:1089680081003700e20f500003003200e30f50008f
:108978007d003a0028003700324090000058a300dc
:1089880079003200f208900002109000808f5000a9
:1089980075003600224090000064a0002041980035
:1089a80071c1b300906680004158980092668000bb
:1089b8000258900001cfb30001406000f040b300be
:1089c8000059980068003700324090000058a30012
:1089d80065003200f208900002109000808f50006d
:1089e80061003600224090000064a00020419800f9
:1089f80071c1b3009066800041589800926680006b
:108a08000258900001cfb30001406000f040b3006d
:108a18000059980054003700225890000004e000e4
:108a280014003500324090000058a3004e00320078
:108a3800f208900002109000808f50004a00360023
:108a4800224090000064a0002041980071c1b3004a
:108a58009066800041589800926680000258900005
:108a680001cfb30001406000f040b3000059980006
:108a78003d003700324090000004a00030419800cb
:108a880091668000015890000040e80080589800e6
:108a980035003700324090000004a00030419800b3
:108aa80091668000015890000040e80080589800c6
:108ab8002d00370000802300808f50000d003a0001
:108ac800234090000054a000a041980011c1b300b9
:108ad8009066800041589800926680000258900085
:108ae80001cfb30001406000f040b3000059980086
:108af8001d003700a34090008140e800ffc06000df
:108b08002340900002ceb300024060000140700094
:108b1800a041980091668000214090007f0060008d
:108b2800f30f500010003400214090000064a000b2
:108b3800a040980031c1b300906680004158980069
:108b4800926680000258900001cfb3000140600097
:108b5800f040b30000599800f00f200070248800fe
:108b680020002000502488002df707008cc4bf0087
:108b78000028a3002c0032008ac4bf000028a300ec
:108b8800290032004000200050248800336780000c
:108b98000300e0001e003200230090000000e00007
:108ba80018003200a00090000100e000150032001b
:108bb8000230200005102000f4ceb30051089000c8
:108bc80002006000820f500002003200850f500042
:108bd80006003a00310090000000e0000300320077
:108be800310090000000e900b0009800314090008a
:108bf80004406000b0409800910078000100e00057
:108c0800eeff3a00930178000300e000e2ff3a002b
:108c1800d60ca900d62ca900d64ca900d66ca90060
:108c2800d86cef00fef607008cc4bf000018a30044
:108c38004c0032008ac4bf000018a300490032006b
:108c4800d68ca9009366800033589000634060007a
:108c5800e14f50003f003200a34090008140e800ff
:108c6800ffc060002340900002ceb30002406000c5
:108c780001407000a041980091668000214090005a
:108c88007f006000f30f5000320034008e44e20091
:108c980002003d0000c2b300c05898008ec4bf0057
:108ca8000058a3000300320011c2b3009066800090
:108cb800415898008ec4bf000048a300030032004a
:108cc80021c2b30090668000415898008ec4bf004e
:108cd8000038a3000300320031c2b3009066800060
:108ce800415898008ec4bf000028a300030032003a
:108cf80041c2b30090668000415898008ec4bf00fe
:108d08000018a3000300320051c2b300906680002f
:108d1800415898008ec4bf000008a3000300320029
:108d280061c2b30090668000415898009166800047
:108d3800214090000064a000a04098009266800046
:108d48000258900001cfb30001406000f040b3002a
:108d580000599800f00f200070248800200020009f
:108d6800502488004f03be004f02be004f01be00d2
:108d78004f00be003600f90000400600881f78004a
:108d88000000eb008008880011a1a90010c1a9000b
:108d98000111200091407800f2ccb30082c060003d
:108da8000144a0008000fd0010e1b7008000fd0034
:108db8001061a9001021a9003008880011e1a8005d
:108dc80080007800e7d3290066002000a5d229009a
:108dd80004c4290063d1290082bb200061807b0084
:108de8000608780061807a000408780061807900bc
:108df800020878008180e800f48f5000f7ff3a00fd
:108e0800f0032000900c8800e00c8800300d8800ea
:108e1800800d8800d00d8800200e8800700e880014
:108e2800c00e8800100f8800d5c6bf0008ccb3005c
:108e3800084060002041b300d5e6b70092a1a90020
:108e480000a0260081012000671a0700dac6bf00cb
:108e5800084060003041b300dae6b7009ca1a900e1
:108e680000a02600810120005f1a0700d3c6bf00ba
:108e7800084060004041b300d3e6b700a6a1a900ae
:108e880000a0260081012000571a0700dbc6bf009a
:108e9800084060005041b300dbe6b700b0a1a9006c
:108ea80000a02600810120004f1a0700d2c6bf008b
:108eb800084060006041b300d2e6b700baa1a9003b
:108ec80000a0260081012000471a0700dcc6bf0069
:108ed800084060007041b300dce6b700c4a1a900f7
:108ee80000a02600810120003f1a0700cdc6bf0060
:108ef800084060008041b300cde6b700cea1a900cc
:108f080000a0260081012000371a0700c1c6bf0053
:108f1800084060009041b300c1e6b700d8a1a9009d
:108f280000a02600810120002f1a0700c0c6bf003c
:108f3800084060003042b300c0e6b700e2a1a900d3
:108f48000001eb009208880013a1a90012c1a90032
:108f580012c1bf00f1ccb300014060000044a00082
:108f680012e1b7001221a9005208880013e1a800f5
:108f78009500a80070c0b300a860b7004f0478003f
:108f880000000600889fbe00800478000104780075
:108f98000000e00005003a0020d52900ad180700c0
:108fa80008007800050a07000d00370000d72900df
:108fb800a81807000000eb00004088001040880057
:108fc8002040880001a62e003164880030408800c7
:108fd80040408800504088000004780002003700b4
:108fe800e90f540039003e007a40b900418820005a
:108ff8000002eb0004b078008081e800d20720006e
:1090080082b178006401400004b178006601400034
:10901800a500200005b178006801400004b178007f
:109028000501400004b178006c01400004b17800eb
:10903800ee0140004201200082b17800700140003a
:1090480005b178007201400004b17800f4014000d5
:109058000208200082b178007601400004b178004f
:109068007800400082bb200002b0780066005400ff
:10907800e30f500003003e000020200080b178007c
:109088000e00370064005400e10f500006003e0057
:109098007a40b900740040008001eb00428820004b
:1090a80003307900050037007a40b90074004000a9
:1090b800030820004288200003307900ea004400b9
:1090c80080bb200083e007000d0037006a005400d1
:1090d8004300dd00829820008001eb000330790016
:1090e8008080e80083307900e401400051002000ce
:1090f800813179006600400041012000013079008b
:109108000804e800fa0f540002003e00e18f540002
:10911800b3ff320000d929004e1807004f04be00e3
:1091280000000600889fbe008a9fbe008c9fbe007c
:10913800800578000006eb00ed0120007a60b90098
:1091480042882000800441000d0478000005eb00ef
:109158000b00e00004003200880078001900780055
:109168005ce0070003003700080078000ee0070005
:10917800800c78000a05e8008984e8000804e80003
:10918800ed0f5500f2ff3a000c06e800ed864600a8
:10919800ea0f5600e9ff3a000006eb000d0a20002e
:1091a800c360dd0080982000808440000d047800b2
:1091b8004a0020000b00e00004003200880078001c
:1091c8001900780043e00700030037000800780022
:1091d800f5df0700800c78000a05e9008984e800bb
:1091e8000804e8000a00e000f2ff3a000c06e80074
:1091f800e4864600f10f5600e9ff3a000b00e00054
:1092080016003200004080008d00780031e0070031
:109218008d00e800104080002ee007008d80e800f7
:10922800204080002be00700e38046003064800087
:1092380028e00700e48046003040800025e0070071
:10924800e58046004040800022e00700e6804600b6
:10925800504080001fe00700150037000d0078001f
:10926800d1df0700004088000d00e800cedf0700ce
:10927800104088000d80e800cbdf07002040880000
:1092880063804600c8df07003064880064804600b9
:10929800c5df07003040880065804600c2df070050
:1092a8004040880066804600bfdf070050408800c5
:1092b80077805600fb17070070d92900e5170700cb
:1092c8004f06be004f05be004f04be00000006005a
:1092d800d0da2900df1707000000eb0091ff070034
:1092e80000d92900db1707000000060070dc290000
:1092f800d8170700100020008aff0700a0dd29000a
:10930800d41707000000060040882000000006006f
:1093180080982000000006003064800000000600ed
:10932800889fbe008a1f7800000578001208e200b6
:1093380019003a002b1507001000e00010003a0051
:1093480028150700001490000800e0000c003a00ff
:1093580020de2900bf170700100020009040880079
:1093680078408800884088000800780013090700c2
:109378008800780008007800960407000600370087
:109388001208e20004003a00200020009c150700a3
:10939800100020008c0437001028ec000f1507007f
:1093a800200090000000e0005a003a000b1507006a
:1093b800100090000000e00056003a000b1507006e
:1093c800300890000000e000080032007140800082
:1093d8008100e800b2012000110009008280d80055
:1093e8008000fd0070408800f4080700ff140700a3
:1093f800200890000000e0000f003200704080005c
:109408000000e00003003a00a0012000704088003e
:10941800020037000000e9007040880071408000b9
:10942800b2012000110009008280d8008000fd00f0
:1094380070408800e10807000ec8bf00f314070059
:10944800e814070041062000908f100008003a0039
:10945800e2140700300090000000e00004003a0029
:1094680071408000c7fe0700500020006415070007
:10947800dc140700c1122000908f100008003a0089
:10948800d6140700b00090000100e00004003a0084
:1094980010002000bbfe0700a000200058150700a0
:1094a800d0140700b000900040062000808f5000c4
:1094b80009003a00c91407001000e00006003a004d
:1094c8008aff07001000200060408800500020003c
:1094d8004b1507005f003700c014070030009000ec
:1094e8000000e00003003a0060408000e10f5000f7
:1094f800020032000a00e00056003a00a0df29000e
:10950800541707000000eb00904088006040880076
:109518002d043700b1140700200090000000e0007f
:109528004b003200b1140700400890000000e00032
:10953800290032000208ec00630060001040880037
:10954800e10f50000d00320005003900e20f500015
:1095580011003200e30f50001d003a0015003700db
:1095680010e129003b17070041e2a90042c2a90007
:109578004302a80041e2a8001700370020e22900b2
:109588003417070041e2a90042c2a9004302a9001a
:1095980041e2a8001000370030e329002d1707002a
:1095a80041e2a90042c2a8004302a80041e2a80083
:1095b8000900370040e429002617070041e2a90006
:1095c80042c2a8004302a90041e2a80002003700f5
:1095d80050e529001f170700841407006008900051
:1095e8000000e0000a003200860ce20005003a00a4
:1095f80000a62e0030648800a0e629001517070091
:1096080003003700862cef0090e8290011170700a7
:1096180076140700001090000000e0000d003200f2
:109628000408ee000408b7004f00de0061001000d7
:10963800204088000300320030ea2900051707009f
:1096480004003700a0ec29000217070001003700ca
:109658006214070070408000e90f5000c1023e000c
:109668005e140700200090000000e000bb003200fc
:109678005e140700500090000000e00007003a0068
:1096880058140700d000900020032000808f50005d
:10969800190036001008ab0017003a00704080002f
:1096a8007a00b9007201400043882000e280790006
:1096b800700c2000808f500003003c000100e8007f
:1096c80000b179000200370020002000cc14070008
:1096d80050ef2900df160700704080007a00b900bb
:1096e800720040004288200060007900531707008c
:1096f800d0ef2900d71607003c140700700090002f
:109708000000e00007003a0036140700f00090005f
:1097180020032000808f5000190036001008ab008d
:1097280017003a00704080007a00b90072014000ca
:1097380043882000e280790080f32f00808f50005a
:10974800030034000100e90000b17900020037008d
:1097580020002000aa14070050ef2900bd160700ba
:10976800704080007a00b9007200400042882000f2
:109778006000790031170700d0ef2900b5160700ff
:109788001a140700400090000000e00007003a00ab
:1097980014140700c000900020032000808f5000a0
:1097a800180036001008ab0016003a007040800020
:1097b8007a00b900f000400042882000610079007a
:1097c800f30f500003003c000000e80080307900ef
:1097d80002003700200020008914070000f029004b
:1097e8009c160700704080007a00b90070004000a5
:1097f80042882000600079001017070010f1290046
:1098080094160700f9130700600090000000e000bc
:1098180007003a00f3130700e0009000200320003f
:10982800808f5000180036001008ab0016003a0070
:10983800704080007a00b900f000400042882000a3
:1098480061007900e10f5000030034000000e900d6
:1098580080307900020037002000200068140700db
:1098680000f029007b160700704080007a00b900dc
:10987800700040004288200060007900ef16070061
:1098880010f1290073160700d8130700200890006c
:109898000000e00016003200734080000002eb0078
:1098a8007a18b900680040004288200060007900fa
:1098b8000000e00001003a00140020007a18b90006
:1098c8006800400042882000043079000400e0006d
:1098d80003003a0090f129005e16070004003700e3
:1098e800e10f520002003a0000f329005916070060
:1098f800be130700300890000000e0001902320093
:10990800734080000002eb007a18b9006a0040003a
:1099180042882000600079000000e00001003a0061
:10992800140020007a18b9006a004000428820001c
:10993800043079000400e00003003a0070f42900c4
:109948004416070007023700e10f520005023a00eb
:10995800e0f529003f160700020237009f130700b1
:10996800100090000000e000ca0032009f130700ba
:10997800400090000000e00007003a00991307003b
:10998800c000900020032000808f5000180036008f
:109998001008ab0016003a00704080007a00b90049
:1099a800ee0040004288200061007900f30f50006b
:1099b80003003c000000e800803079000200370016
:1099c800200020000e14070050f729002116070078
:1099d800704080007a00b9006e0040004288200084
:1099e8006000790095160700c0f8290019160700cd
:1099f8007e130700600090000000e00007003a00b6
:109a080078130700e000900020032000808f5000aa
:109a1800180036001008ab0016003a0070408000ad
:109a28007a00b900ee004000428820006100790009
:109a3800ea0f5000030034000000e900803079008c
:109a48000200370020002000ed13070050f729001e
:109a580000160700704080007a00b9006e004000d0
:109a6800428820006000790074160700c0f82900b9
:109a7800f81507007040800064005000e10f5000a6
:109a880010003e0059130700600890000000e00035
:109a98000c0032000008ee000008b7004f00de009e
:109aa8006100100000408800e10f500003003a00f8
:109ab80030f92900e71507000200370060fa29008d
:109ac800e415070070408000e10f500010003e00d0
:109ad80046130700600890000000e0000c00320008
:109ae8000608ee000608b7004f00de00610010000f
:109af80030408800e10f500003003a00a0fb290025
:109b0800d415070002003700c0fd2900d115070051
:109b18000e88ed00e10f500010003e0033130700df
:109b2800600890000000e0000c0032000808ee0019
:109b38000808b7004f00de006100100040408800b0
:109b4800e10f500003003a00f0ff2900c11507009b
:109b58000200370020022a00be1507002313070061
:109b6800700890000000e000110032000a08ec00c4
:109b7800670060005040880003003200e10f500089
:109b880007003a000300370060042a00b1150700f7
:109b98000700370020062a00ae150700040037002a
:109ba800d0072a00ab1507000a88ec000307070056
:109bb8000e130700500890000000e0001a00320061
:109bc800704080007a00b900760040004488200088
:109bd80060017a000201e80033002000801f78004d
:109be800110009000381d8004f00780001307a0085
:109bf800e18f50000700320003003900e28f500067
:109c080009003a0006003700300b2a0091150700ba
:109c180005003700100d2a008e15070002003700d6
:109c2800d00f2a008b150700f012070020089000bb
:109c38000000e0004b013200734080000002eb009e
:109c48007a18b9006c004000428820006000790052
:109c58000000e00001003a00140020007a18b90062
:109c68006c00400042882000043079000400e000c5
:109c780003003a0090122a007615070039013700d0
:109c8800e10f520037013a00a0132a0071150700ae
:109c980034013700d5120700500090000000e000a2
:109ca80007003a00cf120700d000900020032000e0
:109cb800808f5000180036001008ab0016003a00dc
:109cc800704080007a00b900800078004388200046
:109cd80060817900700c2000800f510003003c0067
:109ce8000200e80080b07900020037002000200060
:109cf8004313070060142a005615070070408000bf
:109d08007a00b9004288200062007800cb1507006d
:109d1800d0ef29004f150700b4120700700090001b
:109d28000000e00007003a00ae120700f0009000c3
:109d380020032000808f5000180036001008ab0068
:109d480016003a00704080007a00b9008000780060
:109d5800438820006081790080f32f00800f510034
:109d6800030034000200e90080b0790002003700e7
:109d7800200020002213070060142a003515070070
:109d8800704080007a00b9004288200062007800a4
:109d9800aa150700d0ef29002e1507009312070017
:109da800400090000000e00007003a008d12070014
:109db800c000900020032000808f5000190036005a
:109dc8001008ab0017003a00704080007a00b90014
:109dd8000081e80043882000e2807900900f20008d
:109de800808f500003003c000100e80000b17900ba
:109df80002003700200020000113070060152a0028
:109e080014150700704080007a00b9000080e8004f
:109e1800428820006000790088150700d0ef2900eb
:109e28000c15070071120700600090000000e000a8
:109e380007003a006b120700e000900020032000a2
:109e4800808f5000180036001008ab0016003a004a
:109e5800704080007a00b9008080e80042882000c5
:109e6800610079000000e000030034000000e90010
:109e7800803079000200370020002000e01207003f
:109e880060152a00f3140700704080007a00b900ba
:109e98000080e8004288200060007900671507000c
:109ea800d0ef2900eb14070050120700500890006b
:109eb8000000e00007003a004a120700d0089000ae
:109ec80020032000808f5000190036001008ab00d6
:109ed80017003a00704080007a00b9006401400021
:109ee80043882000e2807900c0072000808f50005e
:109ef80003003c000100e80000b1790002003700cf
:109f080020002000be120700f0152a00d114070017
:109f1800704080007a00b900640040004288200048
:109f28006000790045150700d0ef2900c914070023
:109f38002e120700700890000000e00007003a00a9
:109f480028120700f008900020032000808f50009e
:109f5800180036001008ab0016003a007040800068
:109f68007a00b900e40040004288200061007900ce
:109f78000000e000030034000000e90080307900b0
:109f880002003700200020009d120700f0152a006b
:109f9800b0140700704080007a00b90064004000e7
:109fa800428820006000790024150700d0ef2900be
:109fb800a81407000d120700400890000000e000f8
:109fc80007003a0007120700c0089000200320008d
:109fd800808f5000190036001008ab0017003a00b7
:109fe800704080007a00b900660140004388200074
:109ff800e2807900700c2000808f500003003c0044
:10a008000100e80000b179000200370020002000bc
:10a018007b120700b0162a008e14070070408000db
:10a028007a00b9006600400042882000600079008c
:10a0380002150700d0ef290086140700eb1107006e
:10a04800600890000000e00007003a00e5110700f2
:10a05800e008900020032000808f50001800360090
:10a068001008ab0016003a00704080007a00b90072
:10a07800e60040004288200061007900e10f5000ae
:10a08800030034000000e900803079000200370046
:10a09800200020005a120700b0162a006d1407008d
:10a0a800704080007a00b9006600400042882000b5
:10a0b80060007900e1140700d0ef2900651407005b
:10a0c800ca110700001090000000e00011003200e3
:10a0d800c8110700714080007a09b9007401410075
:10a0e8004888200081804000e100780001317c0030
:10a0f800a0172a0057140700704080007a00b900a2
:10a108007400400060007c00a0140700d0ef290014
:10a1180050140700b311070080109000400620007b
:10a12800808f50000f003a00b0182a004914070029
:10a138000004eb0089892000ae1107008800440064
:10a14800e10c78000804e800fa844400ea0f54009f
:10a15800f9ff3a00a0dd29003e1407000800780046
:10a1680027120700704080006a0450001000200089
:10a17800f00f540014013e009811070020009000d1
:10a188000000e0000c013a009411070090049000d0
:10a198000900e00008013a009411070060089000e7
:10a1a8000000e00011003200090178004340dd00a2
:10a1b80081982000608078000000e00001003a00eb
:10a1c80012002000c340dd00809820008230780013
:10a1d800e10f510003003a00d01a2a001d140700ad
:10a1e80002003700001c2a001a1407007f1107001c
:10a1f800400890000000e0003b0032004340dd00d2
:10a208000080e8008198200060807800e20f50000c
:10a218001b00320005003e000000e000080032008c
:10a22800e10f50002e003a000d003700e30f5000f8
:10a238001b003200e40f500029003a0020003700cc
:10a248004340dd000080e8001200200081982000d3
:10a2580002b07800101d2a00fe1307002200370004
:10a268004340dd000080e8002200200081982000a3
:10a2780002b07800201e2a00f61307001a003700e3
:10a288004340dd000080e800320020008198200073
:10a2980002b07800801f2a00ee1307001200370072
:10a2a8004340dd000080e800420020008198200043
:10a2b80002b07800b0202a00e61307000a00370031
:10a2c8004340dd000080e8000001eb008198200099
:10a2d80002b0780050222a00de130700020037007f
:10a2e800a0232a00db1307003e110700d0009000ce
:10a2f800803e2000808f5000090036004340dd007a
:10a308006401400083982000e280790050a52e0067
:10a31800808f500002003e006a80400000b1790042
:10a3280032110700500090000000e00007003a00da
:10a338002c110700d000900020032000808f5000cf
:10a34800170036001008ab0015003a004340dd0046
:10a358006401400083982000e2807900f0a52e0077
:10a36800808f500003003e000100e80000b1790032
:10a378000200370020002000a1110700f0242a0065
:10a38800b41307004340dd006400400081982000ba
:10a3980060807800fd130700d0252a00ad13070060
:10a3a80010110700f0009000803e2000808f5000c0
:10a3b800080036004340dd00e40040008298200099
:10a3c80061007900eb0f5000020036006a0050006f
:10a3d8008030790005110700700090000000e0004f
:10a3e80007003a00ff100700f0009000200320004b
:10a3f800808f5000160036001008ab0014003a0099
:10a408004340dd00e40040008298200061007900ac
:10a41800e10f5000030036000000e90080307900a9
:10a42800020037002000200075110700f0242a00e0
:10a43800881307004340dd00640040008198200035
:10a4480060807800d1130700d0252a008113070007
:10a45800e4100700c0009000803e2000808f50006c
:10a46800090036004340dd00660140008398200063
:10a47800e280790050a52e00808f500002003e0037
:10a488006a80400000b17900d810070040009000b1
:10a498000000e00007003a00d2100700c00090005a
:10a4a80020032000808f5000170036001008ab00f2
:10a4b80015003a004340dd00660140008398200003
:10a4c800e2807900f0a52e00808f500003003e0046
:10a4d8000100e80000b179000200370020002000e8
:10a4e8004711070040262a005a1307004340dd00a1
:10a4f800660040008198200060807800a313070060
:10a50800d0252a0053130700b6100700e00090007a
:10a51800803e2000808f5000080036004340dd0058
:10a52800e60040008298200061007900ec0f50009e
:10a53800020036006a00500080307900ab10070036
:10a54800600090000000e00007003a00a510070036
:10a55800e000900020032000808f50001600360095
:10a568001008ab0014003a004340dd00e60040004c
:10a578008298200061007900e20f50000300360045
:10a588000000e90080307900020037002000200038
:10a598001b11070040262a002e1307004340dd0048
:10a5a80066004000819820006080780077130700db
:10a5b800d0252a0027130700880078000a007800b1
:10a5c80004000700100020004f0578004f04be006b
:10a5d80000000600e4874700889fbe008a9fbe00ef
:10a5e8008c9fbe008e1f78000006780081bf9f00f8
:10a5f8000005eb008006eb008b9820006e8320009e
:10a60800e10f560004003a000fbc97001a01200021
:10a61800290020000a003700e20f5600030032002c
:10a628000a0478008a047800050037000a0045000b
:10a6380001a120000db078000a0478008a0478008f
:10a648004340dd000080e80060807d00e20f50009c
:10a658002200320005003e000000e0000800320041
:10a66800e10f50008a003a000b003700e30f50005a
:10a6780038003200e40f500085003a0057003700d8
:10a68800561007000801440089804400e100780062
:10a6980001317f007e003700541007008980440094
:10a6a800610078000000e0000800320088004400e3
:10a6b80002a120008001eb00610079000000e000a9
:10a6c80001003a001300200083307900080044009c
:10a6d80002a12000623778006d00370043100700a0
:10a6e80089804400610078000000e0000500320025
:10a6f800880044001000200042812000803079004a
:10a7080080307f000801440043812000e280790006
:10a718000100e0000a0032004340dd006400400010
:10a7280060807d00808f500005003e0010002000f2
:10a7380000317f000100e80000b1790054003700c3
:10a7480008004400418120000db078000d307f00e2
:10a758004f0037002110070089804400610078000d
:10a768000000e00018003200080244004281200086
:10a77800e40179004340dd00e600400061817d008e
:10a78800801f7800110009008281d8004f007800ee
:10a798006400400060807d00808f5000030031001d
:10a7a8001000200000327f0002003700080044003b
:10a7b8000d307f00880044000300e800428120003b
:10a7c8008030790032003700080044000d307f00e7
:10a7d800418120000db078002d00370003100700dc
:10a7e80089804400610078000000e0000800320021
:10a7f8008800440002a120008001eb00610079007c
:10a808000000e00001003a001300200083307900c6
:10a818008801440002a12000630079000000e000e4
:10a828001700320040812000630278004340dd00b9
:10a83800e600400061817d00801f7800110009005a
:10a848000282d8004f0078006400400060807d00dc
:10a85800808f5000030031001000200080317f00fd
:10a8680002003700080044000d307f0088004400d3
:10a878000400e8004281200080307900040037009d
:10a88800080044000d307f00418120000db07800a1
:10a898004340dd00e0817d00e18f510008003a006f
:10a8a80088004400628320000002eb006100790008
:10a8b8000000e00001003a000302780084307900cb
:10a8c8000a05e800f00f55004dff360061832000af
:10a8d80091407800e1c06000c308dd00ecc2bf0011
:10a8e80074cfb3000440600001407000ece2b70090
:10a8f8008183200091407800e1c06000c508dd0038
:10a90800d5c2bf00f2cdb300024060000140700024
:10a91800d5e2b700a183200091407800e1c0600033
:10a92800c608dd00d5c2bf00f5cbb3000540600006
:10a9380001407000d5e2b700c18320009140780043
:10a94800e1c0600081c04000dcc2bf00d3cfb300cb
:10a958000340600001407000dce2b700e1832000a2
:10a9680091407800e1c06000c208dd00dcc2bf0091
:10a97800b6cfb3000640600001407000dce2b700cb
:10a988000184200091407800e1c06000c308dd0028
:10a99800dcc2bf000440600001407000dce2b70088
:10a9a8002184200091407800e1c06000c408dd00e7
:10a9b800dcc2bf00f7ceb300074060000140700062
:10a9c800dce2b7004184200091407800e1c06000db
:10a9d800c508dd00dcc2bf00024060000140700015
:10a9e800dce2b7006184200091407800e1c060009b
:10a9f800c608dd00dcc2bf000540600001407000f1
:10aa0800dce2b7008184200091407800c708dd00af
:10aa1800dcc2bf000074a10001407000dce2b70096
:10aa2800a184200091407800e1c06000ecc2bf0022
:10aa3800e2cfb3000240600001407000ece2b700d2
:10aa4800c184200091407800e1c0600081c04000ce
:10aa5800ecc2bf000340600001407000ece2b700a8
:10aa6800e184200091407800e1c06000e4c2bf00aa
:10aa78000240600001407000e4e2b7000185200058
:10aa880091407800e1c0600081c04000e4c2bf008e
:10aa98000340600001407000e4e2b7002185200017
:10aaa80091407800e1c06000c208dd00e4c2bf0048
:10aab8000640600001407000e4e2b70041852000d4
:10aac80091407800e1c06000c308dd00e4c2bf0027
:10aad8000440600001407000e4e2b7006185200096
:10aae80091407800e1c06000c408dd00e4c2bf0006
:10aaf8000740600001407000e4e2b7004f077800ab
:10ab08004f06be004f05be004f04be004f00b10007
:10ab1800000006000f0ab000889fbe008a9fbe0092
:10ab28008c9fbe008e1f78000004eb0049fa2f00ae
:10ab3800898447002f0f070088004400e0b478009c
:10ab48000804e800ea0f5400faff3a002b0f070048
:10ab580080c0eb0090cf100008003200c042800097
:10ab68000000e000070032000000e900c042880051
:10ab7800124c8000b29f9f0002003700e0012000c5
:10ab8800c0428800190f070010009000e10f500024
:10ab980005003a008000eb007008e20001003a006e
:10aba8008000780081438800100f07002000900083
:10abb800e10f500005003a008000eb006e08e2004b
:10abc80001003a00800078007143880050408000fe
:10abd800e10f5000060036000000400043f52f004a
:10abe8008f814100030040005f929700242898005d
:10abf8000005eb00a589200095a79f004e8820003e
:10ac08000a0678004bfa2f008b85470088892000b8
:10ac180088a79f00a9862000f99f9f00e0c5200013
:10ac2800e09f9f00a1002000d19f9f00a2852000e7
:10ac3800c29f9f00ed8820001fa4970014002000e9
:10ac4800980f120008003a00e40e07000010900068
:10ac58000000e00004003200e40e0700100090003d
:10ac68000000e0000b003a0025002000988f120039
:10ac780013003a00d90e0700001090000000e00011
:10ac88000f003200d90e0700200090000000e000fd
:10ac98000b0032006f9c97001800be00420620008f
:10aca8000300200024d607000001be00400f9800d2
:10acb800df9897000200780086d907003000370037
:10acc8008d047800100020009d0f100019003a0034
:10acd800980f100004003a00c40e070010009000fe
:10ace8000000e0000a003a0011002000998f1000cf
:10acf80010003a0022002000980f11000d003a00c1
:10ad0800ba0e0700200090000000e00009003200a1
:10ad18005f98970024d9070080007800400f9800ba
:10ad2800400620000008b800ef9997008089be000f
:10ad3800130037001900e0000f003a00240020003b
:10ad4800980f120003003a0070438000e10f500092
:10ad58000600320015002000988f120006003a0005
:10ad680080438000850f500003003a004f9c9700f5
:10ad7800980d780002003700cf9c97009b0c780054
:10ad8800e90f550031003e00100020008a00dd0068
:10ad9800010078000003b20009003a0001007800c1
:10ada800003cb20017003a006f80600027003200b4
:10adb8009b0078000fa097001084500028003700ef
:10adc80000408000e10f500008003a007f90970093
:10add800ef909700010050002200200011000900a8
:10ade8000200d800000478001d0037009b0178009d
:10adf8000fa197009280510000f82f0000844000b6
:10ae0800170037009b0278000fa2970014805200a9
:10ae18006300b900904388007f9c97001801780070
:10ae28000200500033002000110009000300d80080
:10ae380000014100a2438800020c780011000900bb
:10ae48000301d80000047800050037001b007800d3
:10ae58008fa497001904500070272a00fd100700de
:10ae680050408000e10f5000090036000080e800e3
:10ae78008a0f500006003a008a00450040fa2f0069
:10ae880000804700e10078003047800000845000cf
:10ae98008e027800ae009000810f5400020034004a
:10aea80081015400050037000100ea008001eb0031
:10aeb800800f540001003d0081014400e90f550056
:10aec80011003a00a04b80000098b9006109b90050
:10aed8004f19de0003002000020140008381480072
:10aee8008381d1000281d300004c80006a00b90040
:10aef800cf80de000201400083814800c23f9f00ee
:10af0800d33f9f000a00370041f52f008f80400093
:10af18000c824000350190000299b9001508900094
:10af28006a00b900cf80de00001a41000192490092
:10af3800c2f72f000f0141008c00410043f52f009c
:10af48008f8141000c8041001002be008488be0041
:10af58000a05e8009fa29700fa82420095a79f0081
:10af68007a074700640646008b85e8000fa497001f
:10af78007a04440088a79f00ff9c97008984e80012
:10af8800f99f9f006f98970064004000e09f9f0022
:10af9800df9897008100e800d19f9f00cf99970024
:10afa8008381e800c39f9f00fa864600ea0f550098
:10afb80021ff3a004f809700df8097002f8397008a
:10afc800bf8397000002430081824b0094af9f002b
:10afd800a5af9f000600500087805800b0af9f00c3
:10afe800c1af9f000f8097009f8097001201be009d
:10aff8000004410081844900d8af9f00e9af9f0059
:10b008000202500083825800f4af9f0085b79f006a
:10b0180006024000878248000204520083845a00d6
:10b0280098b79f00a9b79f000202420083824a0096
:10b03800b4b79f00c5b79f0006005000878058002e
:10b048000202400083824800d4b79f00e5b79f0002
:10b058000200500083805800f0b79f0081bf9f0016
:10b068008006eb0065d1290085af9f00e8c5200068
:10b07800f8a79f0049f52f008f844400e9a79f0097
:10b088004c882000a0d22900d0a79f00e1d3290036
:10b09800c1a79f000a08e2001c003200e18f560099
:10b0a8000b00320005003900e28f56000d00320017
:10b0b800e38f560037003a000f0037007fb1970042
:10b0c8008fb99700a22f9f00b32f9f003100370040
:10b0d8005fb29700efb29700c42f9f00d52f9f0053
:10b0e8002c0037003fb49700cfb49700e82f9f009b
:10b0f800f92f9f00270037001fb09700afb09700c7
:10b1080080379f0091379f00220037003040800031
:10b11800e10f50000e003a000d00e000030032007d
:10b12800e18f56000a003a00050037007fa9970012
:10b138008fb19700a22f9f00b32f9f000400370004
:10b148005faa9700efaa9700c42f9f00d52f9f00f2
:10b1580040408000e10f50000e003a00e28f560098
:10b1680003003200e38f56000a003a00050037005a
:10b178003fac9700cfac9700e82f9f00f92f9f00b6
:10b18800040037001fa89700afa8970080379f00da
:10b1980091379f004c0090001e0020000000e00046
:10b1a800010032000087eb006c0090000000e00016
:10b1b80085003a004fa197009200780063002000b4
:10b1c800918f110002003200600020008008780092
:10b1d800e98f560005003a0012c1bf00f1ccb30058
:10b1e800014060000044a00012e1b7005fa2970090
:10b1f800140078000c0578007c019000017d200087
:10b208000191b900020878005c0090000000e0009d
:10b2180030003a001c0090006a00b900cf80de00c0
:10b22800efa297001501be00820f5000838f5800cf
:10b2380002003d00808abe00060037006000100052
:10b24800e0801800800f5100818f590001003d00f7
:10b25800808abe001a0078006a00b90088bb200006
:10b2680000044400cfc4de006173b9001502780001
:10b278000431b8001500900000b0b9000300400088
:10b2880007a2b900840140000801410089814900f2
:10b29800c057210001002000800f5100818f590004
:10b2a800020034000001be0006003700391f2000ec
:10b2b800890f5100e08f590002003c00421f200016
:10b2c800030020008fa8970011007800020878007a
:10b2d800e0003700e10f5000de003a00ffa59700bc
:10b2e8006173b900efa19700130278000431b80028
:10b2f800efa297001500900000b0b90003004000cd
:10b3080007a2b900840140003b044100ab84490016
:10b31800888dbe001c0178009c0390000700410046
:10b32800863e20000680b900043e29004500200022
:10b338000000420081804a00070151000691b900cf
:10b348000201420083814a00800f5400818f5c0013
:10b3580002003400808dbe0004003700820f5400c4
:10b36800838f5c0001003d00828dbe001b00be0083
:10b378000247260083002000820f5000838f580068
:10b3880002003400828dbe0007003700f3342c0021
:10b39800830f5000e08f580003003c0000352c005c
:10b3a80001002000808dbe000faa970014047800c9
:10b3b8001b00be0042062000030020005ed40700e8
:10b3c800000c7800a3003700e10f5000a1003a00fc
:10b3d800cfa297001500780061c02100908f10005f
:10b3e8000100320001087800e98f560004003a0095
:10b3f80012c1bf00f1ccb3000140600012e1b700f8
:10b40800aca79f000c099000803e20000091b90075
:10b41800cf91de0000402200410f200055d40700e4
:10b428000005be00dfa49700190078000a0878001c
:10b438005c0090000000e00039003a001c00900019
:10b448006a00b900cf80de00efa297001501be00a8
:10b45800820f5000838f580002003d00808abe0092
:10b468000600370060001000e0801800800f5100cf
:10b47800818f590001003d00808abe002fa49700eb
:10b4880018007800420620000280b90008712200e6
:10b4980000044400cfc4de006573b900cfb3de00fa
:10b4a800150278000431b8001500900000b0b9000a
:10b4b8000300400007a2b9008401400008024100cf
:10b4c8008982490000e2240001002000800f520018
:10b4d800818f5a00020034000002be0004003700c9
:10b4e800e00f5200e08f5a0001003d006022b800d2
:10b4f8008fac9700190478000a20b80005d1b9006c
:10b50800010141000ba2b9008400410002e22400bd
:10b518000300200017d40700000c78004d00370006
:10b52800e10f50004b003a007fa09700b0a79f00a2
:10b538006173b900efa09700110278000430b800d9
:10b54800efa197001301900002b1b9000101410079
:10b5580007a2b90084004100420120000300200036
:10b56800f5d307007fa2970034044000a484480064
:10b57800088abe00afa297001501780095039000d5
:10b5880007004100260320000680b900047122004c
:10b59800050020000000420081804a000701510098
:10b5a8000691b9000201420083814a00800f5400cd
:10b5b800818f5c00030034007fa49700008cbe00dc
:10b5c80005003700820f5400838f5c0002003d00a5
:10b5d800bfa49700828cbe003fa197001200be0056
:10b5e80002e2240003002000820f5000838f5800dd
:10b5f800030034003fa29700028abe00060037000d
:10b60800e00f5000e08f580003003d00bfa29700f4
:10b61800800aeb00b51278008fac97001904780007
:10b62800bfa09700110278000450b800bfa197008e
:10b638001301900002d1b900010141000ba2b90029
:10b648008400410002e2240003002000c9d307005f
:10b65800000c78008d06e8000faa97000482e80025
:10b6680084af9f00ffa29700e4824200f5a79f00e5
:10b678006fa4970064044400e8a79f007a06460078
:10b68800dfa497008984e800d9a79f004fa09700fe
:10b698000080e800c0a79f00ea8f56007dfe3a00b0
:10b6a8004f0778004f06be004f05be004f04be008e
:10b6b8000f0ab10000000600881f78000004780017
:10b6c80020292a00e30e07000040eb00304c9800c8
:10b6d800404c9800584890000004a100504c980035
:10b6e80098c8bf00704c9800b2c8bf0000549800ba
:10b6f800ccc8bf0010549800e6c8bf00205498007a
:10b7080000c9bf00305c98001ac9bf00405c9800af
:10b71800a049800002102000110009000200d80092
:10b728002074980034c9bf0030749800704a8000b3
:10b73800110009000200d800407498004ec9bf00eb
:10b7480050749800404b8000110009000200d80096
:10b758006074980068c9bf0070749800104c80002d
:10b76800110009000200d800007c980082c9bf00bf
:10b77800107c980008007800530a0700cd0a0700db
:10b78800c50b070020408000e10f500004003a007c
:10b798008000eb00200020008efb0700020037002d
:10b7a8006000b8008bfb0700dafc07004f04780044
:10b7b8000000060010408000000006003600fa0075
:10b7c800881f78000004780080fc2f000f004000dc
:10b7d80021412a001a000900311878006003b100dd
:10b7e800fa0f54000300360080442a00990e07001f
:10b7f8000f00370060462a00960e07000800780000
:10b80800e20e0700a0c3b3009f0e070000c2b300fa
:10b818009d0e07000800440081fc2f008080400036
:10b8280061807f008b0e0700d0ef2900890e07008a
:10b838004f0478000080fa0000000600801f78009e
:10b848003400f80000002000a0018800cdc2bf002d
:10b858000008a30004003a00cd02a8007e08ec000e
:10b868007008880005003700cd02a900f043800069
:10b878008008b5000000e800700888000a21ef0081
:10b888008500a9003400f9004f0078000040060048
:10b89800881f7800cac2bf004600de006100600051
:10b8a8000084fb00e14f5000ab003a00320be2008d
:10b8b800a9003a0000402900660e0700a059800040
:10b8c800b20e0700c0402900620e07007300a900ed
:10b8d8000080eb004016880080168800c01688009b
:10b8e8000017880040178800801788000000eb00c8
:10b8f80060168800a0168800e016880020178800c7
:10b9080060178800a0178800a05980006101b8005e
:10b9180021022000810f5100e08f59008c003e0069
:10b92800026001002200370024003700260037009b
:10b93800280037002a0037002c0037002e00370077
:10b948003000370032003700340037003600370047
:10b95800380037003a0037003c0037003e00370017
:10b9680040003700420037004400370046003700e7
:10b97800480037004a0037004c0037004e003700b7
:10b988005000370052003700540037005600370087
:10b99800580037005a0037005c0037005e00370057
:10b9a8006000370062003700640037006600370027
:10b9b800f0c2a900f4c2a80065003700f0e2a900af
:10b9c800f4e2a80062003700f102a900f502a8001d
:10b9d8005f003700f122a900f522a8005c003700bb
:10b9e800c8a2a900cca2a80059003700c882a900a3
:10b9f800cc82a80056003700c842a900cc42a80053
:10ba080053003700c822a900cc22a80050003700f4
:10ba1800c802a900cc02a8004d003700c902a9003d
:10ba2800cd02a8004a003700c942a900cd42a800ab
:10ba380047003700c962a900cd62a800440037005a
:10ba4800c982a900cd82a80041003700c9a2a90077
:10ba5800cda2a8003e003700e862a900ec62a80069
:10ba68003b003700d902a900dd02a80038003700e2
:10ba7800d922a900dd22a80035003700d942a90043
:10ba8800dd42a80032003700d962a900dd62a800b3
:10ba98002f003700d1a2a900d5a2a8002c0037009a
:10baa800d1c2a900d5c2a80029003700d822a90010
:10bab800dc22a80026003700d842a900dc42a800f2
:10bac80023003700d862a900dc62a80020003700f4
:10bad800d882a900dc82a8001d003700d8a2a900de
:10bae800dca2a8001a003700d8c2a900dcc2a8004e
:10baf80017003700d8e2a900dce2a80014003700dc
:10bb0800e802a900ec02a80011003700e822a90009
:10bb1800ec22a8000e003700e002a900e402a80009
:10bb28000b003700e022a900e422a8000800370033
:10bb3800e042a900e442a80005003700e062a9003d
:10bb4800e462a80002003700e082a900e482a800ad
:10bb58000000e800a0598800985988004f04780030
:10bb680000000600f0402900ba0d07000000eb00b5
:10bb7800d0598800e0598800f0598800206a800070
:10bb8800cdfe07000000060000302f00103a8800a4
:10bb98008001eb00233a880053168800931688002a
:10bba800d316880013178800531788009317880046
:10bbb80080cc2f0040168800f0ff290080168800ee
:10bbc80010f02f00c016880002fc2f000217880012
:10bbd80040ff2f0040178800f0c32f00801788000f
:10bbe800c8c2a800c8e2a800a9c6bf0002406000f9
:10bbf8000014a000a9e6b700a8c6bf000240600074
:10bc08000024a000a8e6b700aac6bf000240600052
:10bc1800c040b300aae6b700c3c6bf000240600038
:10bc28007040b300c3e6b700d802a80081c6bf00c1
:10bc380002406000b040b30081e6b700aec0bf006c
:10bc480081cfb300014060005040b300aee0b700c0
:10bc58008220a9008680a9005700a8005720a800c4
:10bc680057c0a80057e0a8007300a800f308880090
:10bc78001fa1a9001ec1a9001ec1bf000044a10048
:10bc88000054a0001ee1b7001e61a9001e21a900f2
:10bc9800a3088800409c2000d00888001fe1a80065
:10bca800a6c6bf0002406000a040b300a6e6b700e9
:10bcb800d1c6bf00024060005040b300d1e6b700d3
:10bcc800500d070050422900620d0700f03f2f0079
:10bcd80060198800601980000080ea0080198800d7
:10bce80021c3bf00c1cfb3000140600021e3b7000a
:10bcf80000ceb3002063b7002043a9002023a8008a
:10bd08002343a80023c3bf007f40600023e3b7009c
:10bd18002343a80022c3bf0031ccb3000140600018
:10bd28000024a00022e3b7002223a9002203a900cf
:10bd3800f0f321002019880021e3a800a04329007e
:10bd4800440d070087ff07001000200000000600d0
:10bd58000600fa00384be2000e003a0066805700f1
:10bd68001d0c07000000e0000a0032006ff8970081
:10bd780038ebb70020452900360d070038cbbf0047
:10bd8800480d070080482900320d070010002000e8
:10bd9800010037000000eb000080fa0000000600f8
:10bda800889fbe0010002000d059880011b92000db
:10bdb80091407800c808dd0092cbbf000080fb00ee
:10bdc800008440008ecbbf00ee4f50000f003200c1
:10bdd80007003e00e44f500098003200e54f500045
:10bde800d1003200e34f5000dd003a007700370001
:10bdf800f24f500065003200f34f5000da00320075
:10be0800ef4f5000d6003a00ae0037001000200077
:10be1800d0598800b04829000e0d0700c030210015
:10be2800800f54004d00320007003e00c030200053
:10be3800800f54000b00320000912000800f540046
:10be48004f003a000c003700c0a02100800f5400ba
:10be580048003200c0402200800f540048003a00d9
:10be680041003700a0492900fa0c07001000200003
:10be7800e0598800bc003700304a2900f50c07005b
:10be88000000eb00005a880080007800e9b8200024
:10be980028b420006b80100060c07c0080707c009b
:10bea8000080fb00b70d070000c2b300f60c0700c6
:10beb800015a80008100e800015a8800e58f50008f
:10bec800f4ff3400104c2900e20c070021b42000d4
:10bed800914078008180fb0043cbbf004800dd0023
:10bee8000100700011002000fad4070041b42000be
:10bef800914078008180fb0045cbbf004800dd0001
:10bf08000100700021002000f2d4070061b4200075
:10bf1800914078008180fb0047cbbf004800dd00de
:10bf28000100700031002000ead407001000200052
:10bf38009dd407009f0d0700200020009ad4070019
:10bf48009c0d07003000200097d40700990d0700ca
:10bf5800c0402900bf0c070083003700604d29004e
:10bf6800bc0c070080003700404e2900b90c0700c0
:10bf78007d003700304f2900b60c07007a003700e3
:10bf880000512900b30c070077003700904be200fe
:10bf980005003a0090512900ae0c070080002000ef
:10bfa800e05988007000370030532900a90c0700b9
:10bfb80090cbbf000080fb00720d0700c040290035
:10bfc800a40c07003c2bef00670037000055290040
:10bfd800a00c0700904be2000f003a0091cbbf0085
:10bfe800ceebb70092cbbf00cfebb700c05629000d
:10bff800980c070092cbbf000080fb00610d070082
:10c0080091cbbf000080fb005e0d0700700120008f
:10c01800e059880006003700f05729008d0c07000a
:10c0280090cbbf000080fb00560d07003c2bef00b3
:10c03800c0402900870c07004b003700e0598000fa
:10c04800e50f500048003a0070582900810c07009d
:10c0580090cbbf0048ebb70091cbbf0049ebb700ce
:10c0680092cbbf004aebb70093cbbf004bebb700b6
:10c0780094cbbf004cebb70095cbbf004debb7009e
:10c088000000eb00005a880088b4200060407c0063
:10c098000080fb003b0d070000c2b3007a0c0700cc
:10c0a800400bec00005a8800e50f5000f7ff340001
:10c0b800c0402900670c070060002000e059880094
:10c0c80029003700e05a2900620c070090cbbf0016
:10c0d80003003200e24f50000a003a000500370022
:10c0e800505c29005b0c070020002000d059880014
:10c0f8000a003700e05c2900560c07003c2bef00d3
:10c1080006003700105f2900520c070090cbbf00d3
:10c118000080fb001b0d07003c2bef00c0402900ee
:10c128004c0c070010003700d05f2900490c0700ad
:10c13800904be20004003a0000612900450c07001a
:10c148003c2bef000200370090612900410c0700ea
:10c15800c04029003f0c070082fe0700020037009c
:10c1680020002000d05988004f04be0000000600bf
:10c1780010002000d059880054cbbf00e14f500078
:10c18800a1003a00554be2009f003a0057cbbf0090
:10c19800d4ebb700006229002e0c070056cbbf0075
:10c1a800e54f50005800320005003e00e24f5000b5
:10c1b80008003200e44f500090003a003500370084
:10c1c800e64f500053003200e74f50008b003a0012
:10c1d8006d003700d06229001e0c07005acbbf0043
:10c1e800f14f500013003a005b4be20026003a0082
:10c1f80090642900170c07005dcbbf000080fb008e
:10c20800e00c07005ccbbf000080fb00dd0c0700e2
:10c21800c04029000f0c07005ccbbf00d0ebb70073
:10c228005dcbbf00d1ebb700a0002000e05988002b
:10c238008e003700f34f500013003a005b4be200ca
:10c2480011003a00b0652900020c07005dcbbf0061
:10c258000080fb00cb0c07005ccbbf000080fb001c
:10c26800c80c0700c0402900fa0b07005ccbbf00d0
:10c27800d2ebb7005dcbbf00d3ebb700d0002000f6
:10c28800e059880079003700d0662900f10b0700d3
:10c2980076003700c0682900ee0b0700a1b5200022
:10c2a8009140780040cdbf00000ce10008003a0042
:10c2b80041cdbf005b4be30005003a00506a2900fe
:10c2c800e40b0700c0002000e05988006700370031
:10c2d80042cdbf00000ce10008003a0043cdbf008a
:10c2e8005b4be30005003a00c06b2900d90b07003f
:10c2f800f0002000e05988005c003700006d29003c
:10c30800d40b070059003700006f2900d10b070034
:10c3180056003700a0702900ce0b0700a1b52000f9
:10c328009140780042cdbf00000ce1000a003a00bd
:10c3380043cdbf005b4be30007003a000180fb00e0
:10c34800900c0700e0712900c20b070020012000b3
:10c35800e05988000c00370040cdbf00000ce10018
:10c3680009003a0041cdbf005b4be30006003a00ec
:10c378000180fb00830c070070722900b50b0700d1
:10c3880030012000e059880000732900b10b070034
:10c39800a1b5200091407800d2cbbf00000ce1008d
:10c3a8000a003a00d3cbbf005b4be30007003a001a
:10c3b8000180fb00730c0700e0712900a50b070042
:10c3c80050012000e05988000c003700d0cbbf0096
:10c3d800000ce10009003a00d1cbbf005b4be30041
:10c3e80006003a000180fb00660c07007072290005
:10c3f800980b070060012000e0598800c040290020
:10c40800940b07001900370021d4200091407800d0
:10c418000104e10015003a0043cdbf00554be3008d
:10c4280012003a0061b520009140780010cab300ac
:10c4380080cf50000b003a0070b5200011c0b30047
:10c4480090cf100009003a00216a8000214890002e
:10c458000004e00005003a00010078001a07070010
:10c4680002003700c04029007a0b070000000600d0
:10c47800e0b8200011c0b30090cf10001a003a00b5
:10c48800402bef0038cbbf00344de3000b003a00df
:10c498000d00370074b520006000b800e5b8200032
:10c4a80060da7a0061004000e0804800820f5000a6
:10c4b800838f5800faff3a00025a8800206a8000e9
:10c4c80001070700080037003f0dab00fbff3200f3
:10c4d800b2698000c3698000e00f5100e08f590005
:10c4e800ecff3a00f5ff370000000600881f7800cf
:10c4f80038cbbf00930a0700004478000004e0002e
:10c508000600320050742900520b07000880fb0017
:10c518001c0c0700c04029004e0b070000e8230050
:10c5280001002000b00c07000880fb004f047800d1
:10c5380000000600889fbe008a1f78000105780069
:10c5480002047800cf91de0038cbbf00a80a0700ac
:10c55800804478000004e0001d0032000080fb00e9
:10c56800080c0700907529003a0b0700a0782900ed
:10c57800380b07003acbbf004a0b07005079290057
:10c58800340b07003ccbbf00460b0700804829004e
:10c59800300b07000000eb00005a88000800e0009c
:10c5a8000900340060407d000080fb00f50b0700a7
:10c5b80000c2b300340b0700400bec00005a88009f
:10c5c800800f5400f7ff3c00f0792900210b070089
:10c5d80000e8230001002000830c07000980fb000d
:10c5e8004f0578004f04be0000000600f60a070059
:10c5f800e10f500005003a00a203200001c220000c
:10c6080050bd2000cbff070014003700ee0a0700da
:10c61800e20f50000e003a0038cbbf008f87e800c9
:10c6280011c0b300e1ff9f008043eb00d662800099
:10c63800050320000002eb001320200092c0b30085
:10c6480011c2b30093e107008f87e90003003700a8
:10c65800b07a2900ff0a070030c0b3000080fb0051
:10c6680000000600881f780038cbbf00344de30077
:10c6780002003a003f0dab0005003a000004e0005c
:10c688000300320037fd07000000eb00d00a070066
:10c69800d0598000e10f50000a0032000300390031
:10c6a800e20f500071033a0065033700e07c29006f
:10c6b800e80a070010002000d05988003c2bef0042
:10c6c8006d033700e059800001002000f70f50008b
:10c6d800e08f580068033e00006001001700370033
:10c6e8003200370044003700600037007900370017
:10c6f8008f00370094003700b5003700ba003700c4
:10c70800bc003700cf0037000a013700410137006d
:10c7180071013700ac013700e40137001602370019
:10c72800530237005d0237008b023700b902370029
:10c73800ec0237001f033700360337000004eb0014
:10c7480078598800206a8000dbfb070000a02600db
:10c7580081012000240c070030c0b3008eebb70025
:10c76800c0c0b3008febb7000800780090ebb700ab
:10c7780050bd2000517d29000f0009003158780074
:10c7880032002000e1b8200050bd200057ff07000c
:10c798000004e00038033a0010002000e059880047
:10c7a80020002000d05988003303370090c0b30020
:10c7b8008eebb70000c1b3008febb700906bef00b2
:10c7c80050bd2000517e290016000900315878001c
:10c7d80032002000e1b8200050bd200043ff0700d0
:10c7e8000004e00024033a0020002000e0598800fb
:10c7f800d05988002003370030c1b3008eebb70052
:10c80800c0c0b3008febb70040c0b30090ebb700d7
:10c8180031c4b3000100780091ebb70000c5b30044
:10c8280092ebb7000100780093ebb700946bef0030
:10c8380050bd2000c17f290014000900315878003c
:10c8480072002000e1b8200050bd200027ff07003b
:10c858000004e00008033a0030002000e059880096
:10c8680020002000d05988000303370040c2b300dd
:10c878008eebb700c0c0b3008febb70030c0b30079
:10c8880090ebb70080c0b30091ebb70050c0b30085
:10c8980092ebb700936bef0050bd20001181290087
:10c8a800160009003158780062002000e1b8200025
:10c8b80050bd20000dff07000004e000ee023a0022
:10c8c80040002000e059880020002000d05988004e
:10c8d800e9023700a0c1b3008eebb700c0c0b300b7
:10c8e8008febb70010c0b30090ebb70030c0b300b7
:10c8f80091ebb70050bd2000818229001500090086
:10c908003158780042002000e1b8200050bd2000d6
:10c91800f6fe07000004e000d7023a0050002000ad
:10c92800e059880020002000d0598800d202370042
:10c9380038cbbf000204200003002000e1b820002b
:10c948003a090700cc02370090c0b3008eebb7005d
:10c9580040c0b3008febb70070c0b30090ebb700d6
:10c9680048cbbf0091ebb70049cbbf0092ebb700b3
:10c978004acbbf0093ebb7004bcbbf0094ebb7009b
:10c988004ccbbf0095ebb7004dcbbf0096ebb70083
:10c99800976bef0051bd2000e083290030000900ab
:10c9a800b0587800a2002000e1b8200050bd200057
:10c9b800cefe07000004e000af023a00700020003d
:10c9c800e059880020002000d0598800aa023700ca
:10c9d80038cbbf000204200003002000e1b820008b
:10c9e80012090700a402370090002000e0598800cf
:10c9f800a1023700a0c1b3008eebb700c0c0b300de
:10ca08008febb70010c0b30090ebb700916bef004d
:10ca180051bd2000f086290016000900b0587800a2
:10ca280042002000e1b8200050bd2000affe070002
:10ca38000004e00090023a0070012000e0598800ec
:10ca48008d023700cecbbf004eebb700cfcbbf0077
:10ca58000042b0004febb70000c1b30050ebb70085
:10ca68008040eb000100780051ebb700c0c0b30074
:10ca780052ebb7000100780053ebb70010c0b300c9
:10ca880054ebb7000100780055ebb70030c0b30095
:10ca980056ebb700d4cbbf0057ebb70080c0b3004c
:10caa80058ebb7000100780059ebb70040cdbf0044
:10cab8005aebb70041cdbf005bebb700d0cbbf004e
:10cac8005cebb700d1cbbf005debb7008000fd0089
:10cad8005eebb7005febb70060ebb70061ebb70048
:10cae8008000fd0060882900da09070040cdbf00fa
:10caf8000080fb00a30a0700c0402900d5090700f1
:10cb080051bd20003089290016000900b05878006e
:10cb180042012000e1b4200050bd200085fe07003e
:10cb28000004e00054023a00b0002000e0598800f8
:10cb380051023700cecbbf004eebb700cfcbbf00c2
:10cb48000042b0004febb70000c1b30050ebb70094
:10cb58008040eb000100780051ebb700c0c0b30083
:10cb680052ebb7000100780053ebb70012c0b300d6
:10cb78000200780054ebb7000100780055ebb700cd
:10cb880040c0b30056ebb7000200780057ebb7007f
:10cb980080c0b30058ebb7000100780059ebb7002c
:10cba800d0cbbf005aebb700d1cbbf005bebb700cf
:10cbb8008000fd005cebb7005debb7008000fd0076
:10cbc800020078005eebb70020c0b3005febb7004f
:10cbd80000c4b30060ebb7000100780061ebb70058
:10cbe80051bd2000a08a290014000900b05878001f
:10cbf80042012000e1b4200050bd20004dfe070096
:10cc08000004e0001c023a0070012000e05988008e
:10cc180019023700cecbbf004eebb700cfcbbf0019
:10cc28000042b0004febb700e0c0b30050ebb700d4
:10cc38008040eb000100780051ebb700a0c0b300c2
:10cc480052ebb7000100780053ebb70010c0b300f7
:10cc580054ebb7000100780055ebb70050c0b300a3
:10cc680056ebb700d4cbbf0057ebb70060c0b3009a
:10cc780058ebb7000100780059ebb700d0cbbf00e4
:10cc88005aebb700d1cbbf005bebb7008000fd00cb
:10cc98005cebb7005debb7005eebb7005febb7008e
:10cca8008000fd0051bd2000f08b2900150009000f
:10ccb800b058780022012000e1b4200050bd2000c7
:10ccc8001cfe07000004e000eb013a0070012000a0
:10ccd800e0598800e8013700cecbbf004eebb70023
:10cce800cfcbbf000042b0004febb70000c1b3008c
:10ccf80050ebb7008040eb000100780051ebb70023
:10cd0800c0c0b30052ebb7000100780053ebb70086
:10cd180010c0b30054ebb7000100780055ebb70022
:10cd280030c0b30056ebb700d4cbbf0057ebb70009
:10cd380080c0b30058ebb7000100780059ebb7008a
:10cd480042cdbf005aebb70043cdbf005bebb70045
:10cd5800d2cbbf005cebb700d3cbbf005debb70015
:10cd68008000fd005eebb7005febb70060ebb7003b
:10cd780061ebb7008000fd00508d290035090700e0
:10cd880042cdbf000080fb00fe090700c04029001b
:10cd98003009070051bd2000208e29001600090027
:10cda800b058780042012000e1b4200050bd2000b6
:10cdb800e0fd07000004e000af013a00e0002000b9
:10cdc800e0598800ac013700cecbbf004eebb7006e
:10cdd800cfcbbf000042b0004febb70000c1b3009b
:10cde80050ebb7008040eb000100780051ebb70032
:10cdf800c0c0b30052ebb7000100780053ebb70096
:10ce080013c0b3000300780054ebb70001007800aa
:10ce180055ebb70040c0b30056ebb70022c0b300d3
:10ce28000200780057ebb70080c0b30058ebb7009a
:10ce38000100780059ebb700d2cbbf005aebb7001e
:10ce4800d3cbbf005bebb7008000fd005cebb70005
:10ce58005debb7008000fd00030078005eebb700d3
:10ce6800020078005febb70000c4b30060ebb700c6
:10ce78000100780061ebb70051bd2000908f2900b8
:10ce880014000900b058780042012000e1b42000e5
:10ce980050bd2000a7fd07000004e00076013a001d
:10cea80070012000e059880073013700cecbbf0025
:10ceb8004eebb700cfcbbf000042b0004febb7003e
:10cec800e0c0b30050ebb7008040eb0001007800f1
:10ced80051ebb700a0c0b30052ebb70001007800d7
:10cee80053ebb70010c0b30054ebb7000100780053
:10cef80055ebb70050c0b30056ebb700d4cbbf001a
:10cf080057ebb70060c0b30058ebb70001007800da
:10cf180059ebb700d2cbbf005aebb700d3cbbf0059
:10cf28005bebb7008000fd005cebb7005debb70082
:10cf38005eebb7005febb7008000fd0051bd20003d
:10cf4800208e290016000900b05878002201200020
:10cf5800e1b4200050bd200076fd07000004e00089
:10cf680045013a0000012000e05988002000200017
:10cf7800d059880040013700cecbbf0020ecb70065
:10cf8800cfcbbf000042b00021ecb70060c3b300b4
:10cf980022ecb7000044eb000004fd0023ecb700ce
:10cfa8000004fd006440500024ecb700080078003d
:10cfb80025ecb700d0cbbf0026ecb700d1cbbf0023
:10cfc80027ecb70035040700cecbbf004eebb70007
:10cfd800cfcbbf000042b0004febb700a0c0b300fa
:10cfe80050ebb7000800780051ebb70060c0b30001
:10cff80052ebb7000800780053ebb700d0cbbf0066
:10d0080054ebb700d1cbbf0055ebb70030c5b30028
:10d0180056ebb70040cfb30057ebb70020c4b300be
:10d0280058ebb70030c0b30059ebb7000004fd005f
:10d038005aebb7005bebb7000004fd0051bd2000c0
:10d04800e090290019000900b0587800e20020009b
:10d05800e1b4200050bd200036fd07000004e000c8
:10d0680005013a0010012000e0598800020137004c
:10d0780038cbbf000204200003002000e1b42000e8
:10d08800fd07070038cbbf00020420000300200082
:10d09800e1b8200065070700f7003700cecbbf00d6
:10d0a8004eebb700cfcbbf000042b0004febb7004c
:10d0b800c0c0b30050ebb7008040eb00010078001f
:10d0c80051ebb70080c0b30052ebb7000100780005
:10d0d80053ebb70010c0b30054ebb7000100780061
:10d0e80055ebb70070c0b30056ebb700d4cbbf0008
:10d0f80057ebb70040c0b30058ebb7000100780009
:10d1080059ebb70042cdbf005aebb70043cdbf0083
:10d118005bebb700d2cbbf005cebb700d3cbbf0053
:10d128005debb70051bd2000809229001c0009006a
:10d13800b058780002012000e1b4200050bd200062
:10d14800fcfc07000004e000cb003a0010012000be
:10d15800e0598800c8003700cecbbf004eebb700bf
:10d16800cfcbbf000042b0004febb700c0c0b30048
:10d1780050ebb7008040eb000100780051ebb7009e
:10d1880080c0b30052ebb7000100780053ebb70042
:10d1980010c0b30054ebb7000100780055ebb7009e
:10d1a80070c0b30056ebb700d4cbbf0057ebb70045
:10d1b80040c0b30058ebb7000100780059ebb70046
:10d1c80040cdbf005aebb70041cdbf005bebb700c5
:10d1d800d0cbbf005cebb700d1cbbf005debb70095
:10d1e80051bd2000509429001c000900b058780057
:10d1f80002012000e1b4200050bd2000cdfc070052
:10d208000004e0009c003a0010012000e05988006a
:10d2180099003700d44bec0000417800d4ebb700fc
:10d22800cecbbf004eebb700cfcbbf000042b00063
:10d238004febb700c0c0b30050ebb7008040eb0025
:10d248000100780051ebb70080c0b30052ebb70083
:10d258000100780053ebb70010c0b30054ebb700df
:10d268000100780055ebb70060c0b30056ebb7007b
:10d278000200780057ebb70040c0b30058ebb70086
:10d288000100780059ebb700d2cbbf005aebb700ca
:10d29800d3cbbf005bebb70042cdbf005cebb70060
:10d2a80043cdbf005debb70051bd2000209629009b
:10d2b80017000900b058780002012000e1b42000ee
:10d2c80050bd20009bfc07000004e0006a003a0003
:10d2d80070012000e059880020002000d059880003
:10d2e80065003700d44bec0000417800d4ebb70060
:10d2f800cecbbf004eebb700cfcbbf000042b00093
:10d308004febb700c0c0b30050ebb7008040eb0054
:10d318000100780051ebb70080c0b30052ebb700b2
:10d328000100780053ebb70010c0b30054ebb7000e
:10d338000100780055ebb70060c0b30056ebb700aa
:10d348000200780057ebb70040c0b30058ebb700b5
:10d358000100780059ebb700d0cbbf005aebb700fb
:10d36800d1cbbf005bebb70040cdbf005cebb70093
:10d3780041cdbf005debb70051bd200020962900cc
:10d3880017000900b058780002012000e1b420001d
:10d3980050bd200067fc07000004e00036003a009a
:10d3a80070012000e059880020002000d059880032
:10d3b8003100370060c0b3008eebb70040c0b30047
:10d3c8008febb70030c0b30090ebb700cecbbf00f7
:10d3d80091ebb700cfcbbf0092ebb70030c1b300e1
:10d3e80093ebb70051bd2000a09729001000090059
:10d3f800b058780062002000e1b8200050bd20003d
:10d408003afc07000004e0001b003a00d5f90700c9
:10d418001900370038cbbf000204200003002000a9
:10d42800e1b420001407070038cbbf000204200035
:10d4380003002000e1b820007c0607000e0037003a
:10d4480038cbbf000204200003002000e1b4200014
:10d458000907070038cbbf000204200003002000a2
:10d46800e1b820007106070003003700b0982900d2
:10d4780078070700bbf9070000e823000100200037
:10d48800d90807004f04780000000600881f7800bc
:10d4980038cbbf00344de30002003a003f0dab002b
:10d4a80005003a000004e00003003200adf907006f
:10d4b8000000eb0046070700f0598000e10f50001c
:10d4c8005000320005003900e20f50006d003200b4
:10d4d800e30f50008d003a0081003700109a2900b0
:10d4e8005c070700100020002fcf070042ebb700b1
:10d4f8004800de0043ebb700200020002acf0700d9
:10d5080044ebb7004800de0045ebb70030002000d0
:10d5180025cf07008080fb008000fd0046ebb700a8
:10d528008000fd00c801de000300780047ebb7006b
:10d5380012c0b300020078008eebb7008043eb0006
:10d54800070078008febb70042cbbf0090ebb70025
:10d5580043cbbf0091ebb70044cbbf0092ebb700c1
:10d5680045cbbf0093ebb7000100780094ebb70000
:10d578000300780095ebb70038cbbf008f87e80031
:10d58800e2ff9f00e6b82000850020000002eb00c3
:10d59800533f200092c0b30011c2b300bddd0700a5
:10d5a8008f87e9000004e00005003a00109d29007b
:10d5b8002807070010002000f059880002003700f3
:10d5c800909d29002307070020002000005a8800aa
:10d5d800e8b8200060407c000080fb00e9070700f5
:10d5e80000c2b30028070700400bec00005a88006f
:10d5f800e70f5000f7ff3400c04029001507070067
:10d6080042003700009f29001207070038cbbf00ef
:10d618008f87e80012c0b300e2ff9f0082437800c2
:10d62800e6b82000850020000002eb00533f2000f0
:10d6380011cab30097dd07008f87e9000004e000f6
:10d6480032003a0020002000f0598800005a880073
:10d65800e8b8200060407c000080fb00c907070094
:10d6680000c2b30008070700400bec00005a88000e
:10d67800e70f5000f7ff3400c0402900f506070007
:10d688002200370020a02900f206070038cbbf008f
:10d698008f87e80011c0b300e1ff9f008043eb00d3
:10d6a800c6c12000450020000002eb00433f2000d7
:10d6b80092c0b30011c2b30076dd07008f87e9007e
:10d6c8000004e00003003a0030002000f059880010
:10d6d8000e003700909d2900de0607000b0037007a
:10d6e80038cbbf000204200003002000e1b820006e
:10d6f800ce0507000004e000040032000080fb00b3
:10d70800a0070700b0a12900d206070000e82300ff
:10d7180001002000340807004f04780000000600cc
:10d72800881f780000072000808f50008400320096
:10d7380012003e0064005000808f500070003200dc
:10d7480009003e0067005000808f500068003200da
:10d758008100390070f92f0000804000e10f50006f
:10d768007d003e007a003700e0062000808f5000e0
:10d778006b0032006e003e00650037000019200083
:10d78800808f50001800320008003e00100720006b
:10d79800808f50006e003200c0f82f0000804000db
:10d7a800e10f50006c003e0069003700301920007e
:10d7b800808f50002700320004003e000080e900fe
:10d7c800808f500064003a001b0037004019200089
:10d7d800808f500035003200f0ff2700808f500006
:10d7e8005d003a005a003700e60f5200e08f5a00f9
:10d7f80059003a004240900038ebb700180020006a
:10d80800d85988000000eb00e0598800f0598800da
:10d8180040a329008f06070038cbbf00a1060700e8
:10d82800804829008b0607008048290089060700e0
:10d83800080078004900370090a6290085060700ef
:10d84800c8f807000000eb00610607001000200080
:10d858004200370038cbbf00344de3003c003a00ab
:10d868003f0dab003a003200b0698000c16980000a
:10d87800e00f5000e08f58003500320052060700d4
:10d88800e10f500003003200e20f500030003a0070
:10d898000300370042f90700100020002f0037006e
:10d8a800f3fa0700100020002c00370038cbbf0027
:10d8b800344de30026003a003f0dab00240032004f
:10d8c800d0698000e1698000e00f5000e08f5800c7
:10d8d8001f0032003c06070000047800e10f5000ea
:10d8e8001b003a0022fa0700080078001b003700e6
:10d8f80000a929005706070010002000170037006c
:10d9080030ac290053060700100020001300370030
:10d9180070af29004f060700100020000f003700e5
:10d92800b0b229004b060700100020000b0037009a
:10d93800a0b629004706070010002000070037009e
:10d9480090b92900430607001000200003003700a3
:10d9580010002000010037000000eb004f047800a1
:10d9680000000600889fbe008a1f780086f807001e
:10d97800e10f50000700320010bc290035060700ef
:10d98800e0bd29003306070020be29003106070044
:10d99800ffff37006000b800a4dc0700e10f50006b
:10d9a80009003a00f0c029002a060700e0bd290056
:10d9b8002806070020c3290026060700ca42e200fd
:10d9c800080035000b00370010bc290021060700ad
:10d9d800e0bd29001f060700d0c329001d06070067
:10d9e800ffff370060c629001a060700a8f70700de
:10d9f800feff37007bcd0700526def000000eb0003
:10da0800e9cd0700a8072000880f50001800320051
:10da18008000eb00100020005aed07008000eb00aa
:10da2800080078002bce07000004e00004003a004c
:10da3800b0c72900070607002cee070014003700be
:10da4800e0c829000306070030ca290001060700bc
:10da58008040eb000140780008cc070011c0b300fb
:10da68000040eb0005cc07000000fe00080037006e
:10da780017ee070050cb2900f60507000000eb0061
:10da8800c9cd07004106070050cc2900f105070061
:10da9800206a800008f707009760a800b1c0bf009f
:10daa800f1c8b300014060000044a000b1e0b70035
:10dab80003cf07009680a800b0ec07000045eb00f4
:10dac8008a4478002a07070032c2bf000008a30072
:10dad80014003200c20507008040780020c5b3005a
:10dae80080cf54000d003a0032c5b300824f550074
:10daf8000a003a0000c0e80080cf5000030032005e
:10db08000145780082447800060037000000fe00d6
:10db18000145780039c5b300020037008a4478000f
:10db28000145780081dd0700a7050700e20f5000d6
:10db380002003a0055fe070004003700a20507005e
:10db4800e10f500001003a00c6fa0700e0598000d2
:10db5800f10f500003003200f0598000e30f50002d
:10db68005d003a00e4a2a90097050700e10f500004
:10db780016003a001b03070030009000c81220006e
:10db8800880f50000500360016030700900f140098
:10db98000200360040012000e0598800deed070051
:10dba8000000e00009003200a40307000004780028
:10dbb800d9ed0700800f54000400360020ce29005c
:10dbc800a405070040012000e0598800ffce0700a7
:10dbd800104078006140600004003200fbce07006e
:10dbe8001040900046edb7000c003700cbc2bf00d4
:10dbf800b12c200091407800c408de004400de000b
:10dc080062006000e1806000010040001100200017
:10dc18008008dd000100780046edb70020c3bf0092
:10dc2800eace07001040780062406000040032002d
:10dc3800e6ce07002040900018ecb7000600370039
:10dc480020c3bf000008a3000300320000188000b2
:10dc58004200de0018ecb700dcce07001040780068
:10dc68006440600004003200d8ce070030409000c5
:10dc780019ecb7000600370020c3bf000008a30056
:10dc880003003200101880004200de0019ecb700d3
:10dc9800b0598000e80f500023003600e4a2a80025
:10dca8000000eb00b059880055030700460507003f
:10dcb800e10f500002003a00206a80002a030700a2
:10dcc80050bd200021cf29000d00090031587800ef
:10dcd80046fa070014003700e4a2a9005903070018
:10dce800c602070000c8eb0080598000e10f500011
:10dcf80003003a00302bef008059800088ed0700c0
:10dd0800b159800060092000808f500001003a005e
:10dd1800e4a2a800b1598000000a2000808f5000ba
:10dd280001003600362bef0000e823000100200038
:10dd3800ad06070063ff37003600f800809fbe007d
:10dd4800829fbe00849fbe00869fbe00881f780009
:10dd58003400f80000002000a0018800362bec00f9
:10dd6800540107004c0207009e020700c812200059
:10dd7800900f1400060036009a0207000010900069
:10dd8800880f5000020036001000200080598800db
:10dd980080598000e10f500004003a00805980004b
:10dda8005fed070080598800080037006000b80060
:10ddb80008f2070018ccbf00e502070019ccbf0025
:10ddc800ce02070046cdbf009002070051f30700be
:10ddd8002023a8008760a9003400f9004f047800c8
:10dde8004f03be004f02be004f01be004f00be00f1
:10ddf8003600f900004006003600f800809fbe009b
:10de0800829fbe00849fbe00869fbe003400f8003b
:10de180000002000a001880040c2bf000018a30035
:10de280040003a006159800000032000808f5000b4
:10de380010003c0060598000f80f500005003c00bd
:10de480062ce07006259800041128000017178009b
:10de580002003700401280001aecb7006702070082
:10de680061598000614078000080fb004012880002
:10de7800280037006159800010032000808f50006f
:10de880007003a005f020700404090000080fb0056
:10de980040128800401280001aecb7001d003700bd
:10dea8006159800020032000808f500009003a004b
:10deb80054020700104090000080fb00b2022000ce
:10dec8000280b90040128800401280001aecb700a6
:10ded800100037006159800030032000808f500007
:10dee80008003a0047020700104890000000d100df
:10def8006f00600040128800401280001aecb700e2
:10df080004003700a00a2000401288004012800058
:10df18001aecb7002c2bec0040c2bf000018a3007d
:10df2800c0ff32008540a9003400f9004f03be004d
:10df38004f02be004f01be004f00be003600f90080
:10df480000400600809fbe003400f800000020005a
:10df5800a00188004142e200130035001600370096
:10df6800b00a20004012880040c2bf000018a30079
:10df7800fbff320040c2bf000058a30006003a0071
:10df88004112800040c2bf000058a300fcff3200cd
:10df9800010078001aecb7002c2bef0040c2a90052
:10dfa8008680a9000400370040c2bf000018a30003
:10dfb800ebff3200efff37003400f9004f00be00de
:10dfc800004006003600f800809fbe00829fbe0019
:10dfd800849fbe00869fbe003400f8000000200029
:10dfe800a001880050c4b300a70407000000000087
:10dff8003400f9004f03be004f02be004f01be00bf
:10e008004f00be003600f900004006003600f80058
:10e01800809fbe00829fbe00849fbe00869fbe0078
:10e028003400f80000002000a001880000d029007a
:10e0380088040700004006003400f9004f03be00c2
:10e048004f02be004f01be004f00be003600f9006f
:10e05800004006003600f800809fbe00829fbe0088
:10e06800849fbe00869fbe003400f8000000200098
:10e07800a0018800b0d029007604070000400600ff
:10e088003400f9004f03be004f02be004f01be002e
:0ce098004f00be003600f90000400600fa
:020000040000fa
:10098000881f780028042000184478000884fb00a1
:100990004544de0091028000ff3ffc0000ceb30022
:1009a0004260b700910288007c3b07009102800002
:1009b000ff3ffc004544dd0042c0bf007f406000b7
:1009c0000840700042e0b700910288004f047800b0
:1009d00000000600889fbe00024478002203200029
:1009e000124178008284fb0006c02000070020002e
:1009f0000080fb008180fb004b02dd00040243000d
:100a0000e0824b004a09dd0002014200e0814a0019
:100a10004019de000001fd0032e0b7000001fd00da
:100a20000000400080804000ca08dd0006804000d1
:100a3000563b0700f34f540008003200f44f5400b7
:100a4000090032008040eb00f24f540008003a00e9
:100a500064006000c200de0005003700680060002e
:100a6000c300de000200370070006000c400de003a
:100a70000900780032e0b7000180fb004f04be009f
:100a800000000600881f7800280320001844780022
:100a900006c02000070020000080fb008180fb00d2
:100aa0004b02dd0004024300e0824b004a09dd00f6
:100ab00002014200e0814a004019de000001fd0011
:100ac00032e0b7000001fd0022042400023b880050
:100ad0000000400080804000ca08dd000680400021
:100ae000800078003e3b0700a5ff07000800780063
:100af00032e0b7004f04780000000600889fbe0077
:100b00008a9fbe008044780032c0bf008085fb0011
:100b10000004eb00030037000804e800e20f540073
:100b20000600320032c1b3008840780009407800e6
:100b3000a8ff0700e10f5000f7ff320006c02000b9
:100b4000070020000982fb004b21dd000201430069
:100b5000e0814b004a40dd0000004100e080490098
:100b60004008de0032e0b700040242000402440004
:100b70004a22dd00060442008004eb000a40200007
:100b80008984e8000884e80008007800ff3a07003c
:100b90008a8f540002003a008004eb000200370004
:100ba000e14f4000f6ff3a000b00780032e0b7005a
:100bb000090078004f05be004f04be00000006008b
:100bc0002f02b000889fbe008a9fbe008c9fbe008f
:100bd0008e1f78000047780032c0bf000080fb0005
:100be000b0af9f008004eb00030037008904e800e9
:100bf000e28f54000700320032c1b3008940780010
:100c00000e40780073ff0700e10f5000f7ff32003d
:100c10000f0037006fd0970032e0b700526da80088
:100c200030002000eb0037006fd0970032e0b700b3
:100c3000522da80010002000e60037006fd097006a
:100c400032e0b70052eda80070002000e10037004c
:100c50000905e800e20f550008003a000005eb0026
:100c6000060037000a05e800e20f550001003a00cf
:100c70000005eb00890f5500ebff320042c1b300c5
:100c80008a4078000e40780052ff07000000e00024
:100c9000f4ff320004c02000050020000e81fb009c
:100ca0004b10dd006103b800a6b79f00b7b79f00e7
:100cb0004a50dd006103b80086b79f0097b79f00d8
:100cc0002fb39700bfb397000400430085804b000b
:100cd0000fb397009fb397000000430081804b0043
:100ce0004008de0032e0b700820541000b004500fd
:100cf0004a00dd00f0af9f00040440000e40780081
:100d00007eff07000000e00001003200524da80005
:100d100052cdbf00a0d79f00520da90010002400a3
:100d2000003b8800880078000080eb00ac3a0700a8
:100d300088007800f00f2000a53a07000884e8003a
:100d40000e80fb00f20f20000280b900e0af9f0090
:100d50008046eb001c00200002c0200003002000a1
:100d6000c2af9f00d3af9f002fb29700bfb29700d2
:100d70000402410085824900c4b79f00d5b79f0097
:100d80000fb397009fb397000600420087804a0088
:100d90004008de0001002000e0b79f00f1b79f008f
:100da000ffab97008283430087bf9f000980450007
:100db0004a00dd00cfa8970001004000a0af9f00cf
:100dc0008d85fb006fa997000b004100f80007001c
:100dd000520dab0002003200520da900070037008f
:100de000880078007e3a0700880078000b007800c1
:100df000773a07000884e8000c06e8008d46e80012
:100e0000e1cf46000d003a006e0037008800780000
:100e10000080eb00723a070088007800f00f200095
:100e20006b3a07000884e8000c06e8000004200084
:100e3000800f560005003200f4ff3700f003200059
:100e4000800f560002003c00ddff370080c6eb003b
:100e5000cbfe0700e1cf4600020032000006eb00a7
:100e6000d7ff37002fd0970052edb7004fe897001b
:100e700032e0b7008fb897000184e80008007800de
:100e8000423a0700804578000886e8000fb99700cd
:100e9000630041003f3a070000047800e1cf4500bd
:100ea000100032000b80fb00efa997000300400008
:100eb000bf000700800f540060ff3a000c04e800f8
:100ec0000c007800313a0700804578000c86e80075
:100ed000080078002f3a070000047800e1cf4500b1
:100ee000f0ff3a007faa9700cfaa970005064200bc
:100ef0004a48dd004fb39700dfb39700000043007e
:100f0000e0804b004008de0032e0b7002fa89700d9
:100f1000203a0700800578002fa897001b3a0700a9
:100f2000804078000a00e00001003a008b05e800ec
:100f3000e38f550002003600522da8000144a100a5
:100f40004fe8970032e0b7000184fb008c00780086
:100f5000080078001e3a07008c0078000b0078002b
:100f60001f3a070030002400003b880084fe070081
:100f70000c007800053a0700800f540004003a0086
:100f80000c007800033a0700808f550005003200fe
:100f90006fd0970032e0b70052eda800700020003b
:100fa0000c003700894078000e407800b5fe07003d
:100fb0006fd0970032e0b700520dd500610060009d
:100fc00004003700f0032000800f56009fff3c0014
:100fd0008eff37004f0778004f06be004f05be005a
:100fe0004f04be002f02b10000000600889fbe0023
:100ff0008a1f780032c0bf000085fb0000c02000bf
:10100000010020004008de0032e0b7000004eb00e1
:10101000030037000804e800e20f54000700320024
:1010200042c1b300884078000040eb0069fe070031
:101030000000e000f7ff3200050037000a007800ea
:1010400032e0b700522da8001000200055003700f4
:101050008044eb000004eb0032c1b300884078000c
:101060000040eb005bfe07000000e00001003a00da
:101070008944e8000804e800e20f5400f6ff3a0053
:101080000904e00015003a00894078000940780022
:101090007cfe070008c02000090020004048de0058
:1010a0000100200032e0b70030002400003b88003f
:1010b000880078000000eb00c9390700880078003c
:1010c000300f2000c23907002dfe07000a0078000b
:1010d00032e0b7000000eb0032003700e1cf5400ef
:1010e00004003a000a00780032e0b7000000eb008c
:1010f0002c003700e2cf540026003a0032c1b30082
:1011000011c0b3000040eb0032fe07000000e00019
:1011100005003a0032c1b300804078002dfe070080
:101120000000e0000f0032000004eb000100370077
:101130000804e8008844780032c1b3008840780091
:101140000040eb0023fe0700e10f500002003a00d0
:10115000e20f5400f6ff3a008940e800e2cf500069
:1011600001003a008040eb000040eb0045fe070024
:101170000040eb0061fe07000000e00001003a00c3
:101180008ffe07000a00780032e0b7000000eb0095
:10119000040037000a00780032e0b70052cda80002
:1011a000600020004f0578004f04be0000000600dc
:1011b000889fbe008a9fbe0000047800e00f2000d8
:1011c000800f54000300360052ada8000080eb00f1
:1011d0003f003700f20f2000110009000284d80000
:1011e000000178000245780032c0bf008085fb0016
:1011f0008004eb00030037008904e800e28f54000c
:101200000700320032c1b300894078000a407800fc
:10121000f0fd0700e10f5000f7ff32000500370036
:101220000b00780032e0b70052cda8000080eb0040
:101230002700370004c02000050020004b51dd00ce
:10124000ca49dd0002004200e0804a00030040007d
:10125000e08048004008de0032e0b70004014100b1
:1012600082814100e13f200083804000f20f200096
:1012700001057800110009000284d8000105fd0075
:101280000920200001047800010078003f390700a0
:101290008880e9008904e900030032008a0f5000c9
:1012a00006003200f7ff3700520da8000b0078004f
:1012b00032e0b7000080eb0005003700080078003e
:1012c000343907008005fd0032e0b7008005fd00dd
:1012d0004f05be004f04be0000000600e487470033
:1012e000889fbe008a9fbe008c9fbe008e1f780024
:1012f0000005780081047800e00f2000808f500006
:101300000300360052ada8005000200080003700d6
:10131000f20f2000110009008280d80080057800bb
:1013200032c0bf000086fb0030002400003b880074
:101330000004eb008b467800030037000804e80047
:10134000e20f54000700320032c1b3008840780039
:101350000b4078009ffd0700e10f5000f7ff3200bf
:10136000050037000c00780032e0b70052cda8002d
:10137000600020006600370004c020000500200047
:101380004b59dd0002014200e0814a004a40dd0085
:1013900000004100e08049004008de0032e0b70074
:1013a0000b804500000044004a00dd008405400039
:1013b00028d5200018447800090078007cff070039
:1013c0008a0f50000a003a00906a800061006000b5
:1013d00007003a000006fd0032e0b7000006fd00fd
:1013e0000004fd0052edb7000004fd004800370086
:1013f0000800780052edb7000d407800bffd0700ef
:10140000000778000000e00005003a000c007800ba
:1014100032e0b700528da800400020003c003700a9
:101420008b0540000a00be00ed380700f80f2000d1
:10143000110009008884d800810478008b007800ae
:1014400009007800e23807004dfd070000000000a9
:10145000000000000b007800ce38070080f79f00e6
:101460008ff097000180fb0008046500880f500092
:10147000050032000c00780032e0b70052eda80001
:1014800070002000220037000b007800bf380700f2
:1014900080f79f008ff097000180fb00808f540041
:1014a000050032000c00780032e0b70052eda800d1
:1014b00070002000160037000b00e800b538070068
:1014c0004880de0080f79f000ff097008080fb00cf
:1014d0004850de00808f5000050032000c0078007c
:1014e00032e0b70052eda80070002000080037007d
:1014f000e03f2000800f570002003a000d407800c6
:10150000affd07000c00780032e0b7000000eb00f0
:101510004f0778004f06be004f05be004f04be00c7
:081520004f00b10000000600bd
:020000040000fa
:10e0a40020c5b30028ecb70010c0b30029ecb700ba
:10e0b40080c0eb00e06280005140980021c7b300ab
:10e0c400e0628000614098000000060000027800d1
:10e0d400e90040000000eb00c3ae20001203200062
:10e0e40031f079000000e800820f5000fcff3a0094
:10e0f4003448900061006000f05488003448900077
:10e104000000d10061006000005588003448900090
:10e114004200de0061006000105588003448900021
:10e124004300de0061006000205588003448900000
:10e134004400de00610060003055880034489000df
:10e144004500de00610060004055880034489000be
:10e154004600de006100600050558800344890009d
:10e164000080fb004700de006055880044489000b2
:10e174006100600070558800444890000000d100a0
:10e184006100600080558800444890004200de0031
:10e194006100600090558800444890004300de0010
:10e1a40061006000a0558800444890004400de00ef
:10e1b40061006000b0558800444890004500de00ce
:10e1c40061006000c0558800444890004600de00ad
:10e1d40061006000d0558800444890000080fb0036
:10e1e4004700de00e055880054489000610060005c
:10e1f400f0558800744890000080fb0000568800a9
:10e20400045090000080fb001056880014509000c9
:10e214000080fb0020568800245090000080fb0002
:10e2240030568800345890000080fb004056880027
:10e23400445890000080fb0050568800b470900051
:10e244008180fb00247090004800dd008080400045
:10e2540061568800d47090008180fb004470900067
:10e264004800dd008080400071568800f470900002
:10e274008180fb00647090004800dd0080804000d5
:10e2840081568800947890008180fb000478900087
:10e294004800dd0080804000915688006460900052
:10e2a400d4eab70074609000d5eab700046890001f
:10e2b400d6eab70000000600881f780044cd0700a6
:10e2c400404090000008a3000400320040cd070045
:10e2d4000048900061006000f05488003ccd0700c5
:10e2e400404090000018a3000500320038cd07001c
:10e2f400004890000000d1006100600000558800d3
:10e3040033cd0700404090000028a30005003200f0
:10e314002fcd0700004890004200de00610060003d
:10e32400105588002acd0700404090000038a30013
:10e334000500320026cd0700004890004300de00af
:10e34400610060002055880021cd07004040900006
:10e354000048a300050032001dcd070000489000ce
:10e364004400de00610060003055880018cd0700cd
:10e37400404090000058a3000500320014cd07006f
:10e38400004890004500de006100600040558800b0
:10e394000fcd0700404090000068a3000500320044
:10e3a4000bcd0700004890004600de0061006000cd
:10e3b4005055880006cd0700404090000004e0005e
:10e3c40005003d0002cd0700004890000080fb00de
:10e3d4004700de0060558800fdcc070050409000e7
:10e3e4000008a30004003200f9cc07001048900094
:10e3f4006100600070558800f5cc07005040900023
:10e404000018a30005003200f1cc0700104890006a
:10e414000000d1006100600080558800eccc07004a
:10e42400504090000028a30005003200e8cc07000b
:10e43400104890004200de006100600090558800a2
:10e44400e3cc0700504090000038a30005003200e0
:10e45400dfcc0700104890004300de00610060003c
:10e46400a0558800dacc0700504090000048a30073
:10e4740005003200d6cc0700104890004400de00ae
:10e4840061006000b0558800d1cc07005040900076
:10e494000058a30005003200cdcc070010489000be
:10e4a4004500de0061006000c0558800c8cc07004c
:10e4b400504090000068a30005003200c4cc07005f
:10e4c400104890004600de0061006000d0558800ce
:10e4d400bfcc0700504090000004e00005003d0060
:10e4e400bbcc0700104890000080fb004700de0012
:10e4f400e0558800b6cc0700604090000008a300f7
:10e5040004003200b2cc0700204890006100600093
:10e51400f0558800aecc0700604090000018a300be
:10e5240004003200aacc0700304890000080fb00b1
:10e5340000568800a6cc0700604090000028a30085
:10e5440004003200a2cc0700404890000080fb0089
:10e55400105688009ecc0700604090000038a3004d
:10e56400040032009acc0700504890000080fb0061
:10e574002056880096cc0700604090000048a30015
:10e584000400320092cc0700604890000080fb0039
:10e59400305688008ecc0700604090000058a300dd
:10e5a400040032008acc0700704890000080fb0011
:10e5b4004056880086cc0700604090000068a300a5
:10e5c4000400320082cc0700005090000080fb0061
:10e5d400505688007ecc0700604090000004e000a4
:10e5e40008003d007acc0700205490000884fb000a
:10e5f40077cc0700105090004800dd000004440070
:10e604006856880072cc0700704090000008a30090
:10e61400080032006ecc0700405490000884fb00d0
:10e624006bcc0700305090004800dd00000444002b
:10e634007856880066cc0700704090000018a3004c
:10e644000800320062cc0700605490000884fb008c
:10e654005fcc0700505090004800dd0000044400e7
:10e66400885688005acc0700704090000028a30008
:10e674000800320056cc0700005c90000884fb00c0
:10e6840053cc0700705090004800dd0000044400a3
:10e69400985688004f04780000000600881f780010
:10e6a4008003eb0007017800e3a92000c5a7200040
:10e6b4000003eb0084a32000a8a5200082004100f1
:10e6c400618079000000e0000400320061807a007b
:10e6d4000000e80080b07a00020037000200410028
:10e6e40006b07a0082004100618079000000e000f9
:10e6f4000600320061007a000000e00003003a00e6
:10e704001000200080307c0002003700020041002d
:10e7140006307c0002004100e0007a00608079004d
:10e72400808f5000010032001700200002004100d9
:10e73400633278000201e800f10f5100dfff3a0074
:10e7440013002000e6a9200085ad200003814100cc
:10e754002402200002024200e4007b0062807a006e
:10e76400808f500004003600e4007b0062807a0051
:10e77400008050000500370003804100e0807a00eb
:10e784002002b00060007b0000805000e50f5000c4
:10e794000100360017002000838041002002200081
:10e7a4000100400060007b0080b07a008301e80033
:10e7b400ea8f5100e5ff3a000700e00005003a0047
:10e7c40090518000e10f400003003200322aec0037
:10e7d400010037009c0007004f0478000000060089
:10e7e400e0a9200000000600c0a7200000000600e9
:10e7f400a0a520000000060000ac200000000600d8
:10e80400c0ae200000000600e062800000000600a8
:10e8140000404000e162800090489800000006003b
:10e82400e10f500005003a00e162800011489000b9
:10e834000014a00090489800060037000000e00093
:10e8440004003a00e1628000114890000014a10025
:10e854009048980000000600e10f500005003a00bf
:10e86400e1628000114890000024a00090489800c4
:10e87400060037000000e00004003a00e162800076
:10e88400114890000024a100904898000000060060
:10e89400e10f500005003a00e16280001148900049
:10e8a4000034a00090489800060037000000e00003
:10e8b40004003a00e1628000114890000034a10095
:10e8c4009048980000000600e10f500005003a004f
:10e8d400e1628000114890000044a0009048980034
:10e8e400060037000000e00004003a00e162800006
:10e8f400114890000044a1009048980000000600d0
:10e904000080fb00b2022000110009000280d80040
:10e91400000178000204e00007003a00e062800091
:10e92400a04090000104a10021409800e062800012
:10e934001240980006003700e0628000a04090007a
:10e944000104a00021409800e06280001240980079
:10e9540000000600e1628000c040980021c3b300bb
:10e96400e0628000314098000000060080007800da
:10e97400504890000008a30002003200a0002000cc
:10e98400a0518800340ae2001d003200716090003a
:10e99400e34f50000e00320003003e00e24f5000ef
:10e9a40011003a000d003700e44f5000050032001a
:10e9b400e54f50000c003a00f0c0b30094ff07008c
:10e9c4000b00370070c0b30091ff07000800370048
:10e9d40030c0b3008eff07000500370010c0b3003d
:10e9e4008bff0700020037000040eb0088ff0700a0
:10e9f400340aed00a051880001003a0084ff0700aa
:10ea0400000006000000e00004003200b05188005d
:10ea140000c0eb00baff070008003700360ae20026
:10ea24000600320000c0eb00b5ff0700360aed0017
:10ea3400b051880001003a00b1ff07000000060051
:10ea44009051800000000600322aef00000006000a
:10ea5400889fbe008a9fbe00004578000204be0065
:10ea64008145780010002000da0107006000b8003a
:10ea7400b0698800c1698800d0698800e1698800ac
:10ea84003f6def000a00780034edb700826a800021
:10ea9400824890008180fb008169880012489000c0
:10eaa4004800dd008080700081698800a2489000e1
:10eab4008180fb0091698800324890004800dd00a5
:10eac40080807000916988000b0078003eedb700eb
:10ead40000472a00e0010700c0482a00de010700c1
:10eae40008007800a8020700904b2a00da0107000a
:10eaf4000a407800ec010700304c2a00d6010700d8
:10eb0400806980004800de009f020700f80f2000a3
:10eb140080698000080060009b020700b04c2a0056
:10eb2400cd010700906980004800de0096020700ce
:10eb3400906980000800600093020700304d2a00ad
:10eb4400c50107003f0da800640020000500200057
:10eb540002d32000011920000a407800f1fa0700ce
:10eb6400100020004f05be004f04be000000060048
:10eb7400889fbe008a9fbe00004578000204be0044
:10eb84008145780020002000920107006000b80051
:10eb9400b0698800c1698800d0698800e16988008b
:10eba4003f6def000a00780034edb700826a800000
:10ebb400824890008180fb0081698800124890009f
:10ebc4004800dd008080700081698800a2489000c0
:10ebd4008180fb0091698800324890004800dd0084
:10ebe40080807000916988000b0078003eedb700ca
:10ebf400604d2a0098010700d04e2a0096010700b4
:10ec04000800780060020700904b2a009201070078
:10ec14000a407800a4010700304c2a008e01070046
:10ec2400806980004800de0057020700f80f2000ca
:10ec3400806980000800600053020700b04c2a007d
:10ec440085010700906980004800de004e0207003d
:10ec540090698000080060004b020700304d2a00d4
:10ec64007d0107003f0da80064002000050020007e
:10ec740002d32000011920000a407800a9fa0700f5
:10ec8400100020004f05be004f04be000000060027
:10ec94000400fa00881f780048d320001844780044
:10eca400804f540049003a0010072000808f500024
:10ecb400040032000000e800808f500043003a0056
:10ecc40011003700140020000500200042d320006a
:10ecd400111920000840780092fa07000040eb0068
:10ece4003fedb70034edb700d0512a005a010700b8
:10ecf400084078006c010700304d2a0056010700d7
:10ed040010002000320037000200e0002f00320023
:10ed1400ea0f5200e08f5a002c003a001202be00a3
:10ed2400d4bf9f00e5bf9f00e240900010c8b3002d
:10ed340080cf50000b003a003f4da900b469880011
:10ed4400c569880034cdbf004400200005002000c0
:10ed5400668157003119200072fa07001000200064
:10ed64001b00370020c8b30080cf50000b003a00ce
:10ed74003f6da900d4698800e569880034cdbf00df
:10ed8400440020000500200066815700411920003e
:10ed940064fa0700100020000d0037000140e9006c
:10eda400e14f500009003e003f2da90034cdbf00c3
:10edb400440020000500200066815700211920002e
:10edc40058fa070010002000010037000000eb0093
:10edd4004f0478000080fa0000000600000178006b
:10ede4003f0dab001000320043d320009341780064
:10edf4000304e0000c0032000000e0000a003200ce
:10ee040080698000920f100007003a009200900081
:10ee140090698000808f500003003a0043419800bd
:10ee240010002000010037000000eb000000060085
:10ee340046d3200016437800804f53001d003a004b
:10ee4400f06980000088a3001a00320000a8a30023
:10ee54000b003200316980008100e80031698800cc
:10ee64002200200020032000808f50001200360072
:10ee74003f4da900262def00220020000e00370090
:10ee84003f4da800362def00382def000202be00e2
:10ee94000101780011c8b3000640780006d80700c5
:10eea4000004e000010032003f4da9000081fb0096
:10eeb4000100370012002000020078000000060064
:10eec40046d3200016437800804f53001b003a00bd
:10eed400f06980000088a300180032000098a300a5
:10eee4000b003200416980008100e800416988001c
:10eef4002200200020032000808f500010003600e4
:10ef04003f2da900282def00220020000c0037001f
:10ef14003f2da8000202be000101780011c0b30019
:10ef24000640780026dd07000004e00001003200fe
:10ef34003f2da9000081fb000100370012002000d2
:10ef44000200780000000600881f78008201780023
:10ef540048d3200018447800804f540021003a0020
:10ef6400f06980000088a3001e0032000098a3000e
:10ef74000b003200516980008100e800516988006b
:10ef84002200200020032000808f5000160036004d
:10ef94003f2da9002a2def00220020001200370087
:10efa4008f87e8000041eb00e2ff9f008243780076
:10efb40001037800830278000002eb0084017800ea
:10efc40011c2b3000840780033d707008f87e900e7
:10efd4000004e000010032003f2da9000081fb0085
:10efe4000100370012002000020078004f0478006e
:10eff4000000060046d3200016437800804f5300db
:10f004001b003a00f06980000088a3001800320059
:10f014000098a3000b003200616980008100e800c1
:10f02400616988002200200020032000808f5000a6
:10f03400100036003f2da9002c2def0022002000e7
:10f044000c0037003f2da8000202be000101780029
:10f0540021c0b30006407800d9dc07000004e000ba
:10f06400010032003f2da9000081fb0001003700a0
:10f0740012002000020078000000060046d32000a1
:10f0840016437800804f53001d003a00f069800059
:10f094000088a3001a00320000b8a3000b0032005d
:10f0a400716980008100e8007169880022002000f5
:10f0b40020032000808f5000120036003f2da9004d
:10f0c4002e2def00220020000e0037003f6da80017
:10f0d4003a2def003c2def000202be000101780042
:10f0e40021c8b3000640780073d707000004e0008d
:10f0f400010032003f6da9000081fb0001003700d0
:10f10400120020000200780000000600e14f5000c9
:10f1140004003200f10f2000e24f500006003a00d4
:10f124000300370048cdbf008080fb000200370099
:10f1340049cdbf008080fb0001007800000006007c
:10f14400e14f500004003200f10f2000e24f500064
:10f1540006003a00030037004acdbf008080fb0060
:10f16400020037004bcdbf008080fb000100780017
:10f1740000000600e14f500003003200e24f50004f
:10f1840006003a00030037000100780048edb7009c
:10f19400020037000100780049edb70000000600c6
:10f1a400e14f500003003200e24f500006003a00e5
:10f1b40003003700010078004aedb7000200370071
:10f1c400010078004bedb70000000600606a800083
:10f1d40000000600606a880000000600200020008d
:10f1e4000000060032c2bf0051c4b3000008a300ef
:10f1f40002003200b01180008040780087c0a9006e
:10f204000100fb000000060010022000c01188006d
:10f214000000eb00801188003062a8009011880083
:10f2240031e2a8003342a80087c0a900000006000c
:10f2340087c0bf000068a30004003a0032c2bf00c8
:10f244008000eb000008a300010032001100200040
:10f254000100780000000600881f7800b0407800a4
:10f26400000478000104e000060032000140780048
:10f274000600070038407800804078000004e00071
:10f28400faff3a004f047800000006000000fb007b
:10f29400a01188000000000033c2bf000008a300d2
:10f2a400fdff320000000600889fbe008a9fbe005a
:10f2b400004178000004e0001f003a0000c3b300de
:10f2c400f2ff0700230037000980fb00110009004a
:10f2d4000380d8008000fd0081447800814f5100f4
:10f2e400f9ff39000104e0001a0032008245780079
:10f2f4000b84fb000985fb00110009000a84d80077
:10f304000004780001c3b30001404400dfff07009c
:10f3140008ccb90088c55500a200200011000900de
:10f324000285d800000578008a4478000a04e000c9
:10f3340008003200eeff370049c6b300a3002000e6
:10f3440030c6b300804f5100dfff3600824578009d
:10f35400e7ff37004f05be004f04be000000060063
:10f36400881f78000004e00004003d000044ea0027
:10f37400d0c2b300c5ff0700010037000044780085
:10f3840008407800c8ff07004f047800000006001a
:10f39400889fbe008a9fbe00800078000000e000c5
:10f3a4001e003a0000c3b300b8ff07002100370075
:10f3b4000a712200a2002000811f780011000900b8
:10f3c4000285d80000057800cf0078008a8f5000ad
:10f3d400f9ff39000a00e0001600320081057800c8
:10f3e400110009008a85d8000004780001c3b30025
:10f3f40001404400a5ff070008d4b90088855500e2
:10f40400a2002000110009000285d8000005780040
:10f414000a00e00007003200f1ff3700f07022001c
:10f42400808f5000e2ff3600810578000a712200c7
:10f43400ebff37004f05be004f04be00000006007e
:10f44400881f78000000e00004003d000004ea008a
:10f45400d0c2b3008dff070001003700000478001c
:10f4640008007800caff07004f0478000000060077
:10f47400889fbe008a9fbe008c9fbe000006be000f
:10f48400e00f5000e08f580025003a0000c3b3009d
:10f494007eff07002a003700a2002000030020009e
:10f4a4000a00be0034c407000005be00800f5600e9
:10f4b400818f5e00f8ff3900e00f5000e08f5800a4
:10f4c4001f0032000a01be000c00be002ac407005f
:10f4d4000004be0001c3b300014044006bff0700f9
:10f4e4000a41b80009d0b900030040000bc4b900b8
:10f4f400880140000206560083865e00a2002000b8
:10f50400030020000a00be001bc407000005be0063
:10f51400e00f5000e08f580009003200e9ff370087
:10f524000aa02c00abb92300f09f2c00a1b9230042
:10f53400800f5600818f5e00d7ff3600e1ff370051
:10f544004f06be004f05be004f04be00000006007b
:10f55400889fbe00e00f5000e08f580005003d007a
:10f5640060041000e0841800d0c2b30047ff070015
:10f57400010037000004be000800be00bcff070005
:10f584004f04be0000000600889fbe00800478007f
:10f594004480de006f006000485a2a0060407c000e
:10f5a4003aff07006f80640060407c0037ff07006b
:10f5b4004f04be0000000600889fbe00800478004f
:10f5c4004c00de00485a2a0060407c002fff0700f0
:10f5d4004848de006f00600060407c002bff07009d
:10f5e4004448de006f00600060407c0027ff070095
:10f5f4006f80640060407c0024ff07004f04be005d
:10f6040000000600889fbe008a1f78000004be0028
:10f614004c08de006f0060004a5a2a0060407d00fa
:10f624001aff07004848de00010020006f00600058
:10f6340060407d0015ff07004448de000100200003
:10f644006f00600060407d0010ff07004048de004e
:10f65400010020006f00600060407d000bff070088
:10f664004449dd004c40de0000007100cc48de005f
:10f674006f00600060407d0004ff07004849dd0022
:10f684004840de0000007100c848de006f006000e2
:10f6940060407d00fdfe07004c49dd004440de0073
:10f6a40000007100c448de006f00600060407d000f
:10f6b400f6fe07006f04640068407d00f3fe070057
:10f6c4004f0578004f04be0000000600804078001b
:10f6d40060c6b30080cf50001b003c006640500061
:10f6e40080cf50000400340090cab30000c0400032
:10f6f4000000fb001500370060c4b30080cf500049
:10f7040011003c006640500080cf500004003400db
:10f7140090ccb30000c040000000fb000b00370099
:10f7240090c3b30080cf500007003c006a405000f3
:10f7340080cf50000400340000cdb30000c040006e
:10f744000000fb00010037000000eb000000060091
:10f754006f406000e94f5000030034007043b00074
:10f764000000fb00020037000043b0000000fb0073
:10f774000000060032c2bf000018a30001003200de
:08f784003222a900000006007a
:020000040000fa
:10152800520d00000200000000000000480d0000fd
:101538000600000002000000818201000200000095
:10154800260d00001a000000000000004e0d0000eb
:10155800040000000200000000000000000000007d
:10156800c60c00006000000000000000000e000033
:101578001000000000000000400d000008000000fe
:101588000200000040004100004e0b000100000076
:101598002c0b0000f000000000000000880c000088
:1015a80024000000020000002a754a0076000000ae
:1015b8000000000000ba75004a7600000000000034
:1015c8000000e000010100000000020000ffff0031
:1015d800ffff0000010000001c0c0000420000009a
:1015e80002000000420c00000000000000000000a3
:1015f80000000000000000000000000000000000e3
:1016080000000000ff2710000032ff002710000034
:1016180032ff270010003200ff27100000320000c0
:1016280000000000000000000000000000000000b2
:101638000000000000002a000c2a0c00320a0000fa
:10164800fa000000000000005e0c00002a00000004
:1016580002000000e093040000e093000400e000b2
:1016680093040000e093040000e093000400e0000d
:1016780093040000e093040000e093000400e000fd
:1016880093040000e09304000060ea0000080000f2
:101698003202000000000000ac0c00001a0000003c
:1016a80000000000540d00001000000000000000c1
:1016b800640d0000020000000000000000000000af
:020000040000fa
:1016c80040c2bf0031ceb300014060000024a0003a
:1016d80040e2b7000000eb00101288004322a90086
:1016e80042e2a80042a2a900201288004402a800f1
:1016f80030280700e10f50000b00320005003900c8
:10170800e20f50000d003200e30f500015003a00c0
:101718000f003700a0542a00ce36070042c2a900a5
:101728004302a80011003700b0552a00c936070047
:1017380042c2a9004302a9000c003700c0562a0083
:10174800c436070042c2a8004302a80007003700b9
:10175800d0572a00bf36070042c2a8004302a9009a
:1017680002003700e0582a00ba3607008540a90071
:10177800a9c0bf0081cfb300014060006040b30042
:10178800a9e0b7009540a80041e2a80040c2bf0008
:101798000018a30005003a00c10a20004112880081
:1017a80040c2bf000018a300fcff320040c2bf00c7
:1017b8000058a30004003a004012800040c2bf0055
:1017c8000058a300fcff320000000600c0ca200039
:0417d8000000060007
:020000040000fa
:10f78c001080ba00000006001000ba00000006004d
:10f79c00801f78000500fc0050052000303b8800dd
:10f7ac00a00a2000303b880061e7a80000000000a0
:10f7bc000000000061e7af00feff37004f0078004b
:10f7cc00000006008088bb000000060080c8bb005b
:10f7dc00000006008008bb00000006008048bb004b
:04f7ec000000060013
:020000040000fa
:10f7f000f03fb1000180b10006003500ee030900c2
:10f8000000000000403fb1000180b100fbff3d005f
:10f810001000b000203fb000020035000080090059
:08f820000000000000000600da
:00000001FF
